 archba

 Timestamp is 56d8e6a8 (Fri Mar 04 07:06:40 2016)

 Preferred load address is 00400000

 Start         Length     Name                   Class
 0001:00000000 00019128H .text                   CODE
 0001:00019128 00000010H .text$01                CODE
 0001:00019138 00007502H .text$s                 CODE
 0002:00000000 00000090H .idata$5                DATA
 0002:00000090 00000428H .rdata                  DATA
 0002:000004b8 00000048H .rdata$debug            DATA
 0002:00000500 00000004H .rdata$sxdata           DATA
 0003:00000000 0000057cH .data                   DATA
 0003:00000580 000001c4H .bss                    DATA
 0004:00000000 0000002eH INIT                    CODE
 0004:00000030 00000028H .idata$2                CODE
 0004:00000058 00000014H .idata$3                CODE
 0004:0000006c 00000090H .idata$4                CODE
 0004:000000fc 00000332H .idata$6                CODE
 0005:00000000 000000c8H .rsrc$01                DATA
 0005:000000d0 00001110H .rsrc$02                DATA

  Address         Publics by Value              Rva+Base       Lib:Object

 0000:00000001       ___safe_se_handler_count   00000001     <absolute>
 0001:00000010       _GetOutstandingIoCnt@4     00401010 f   rxdevice.obj
 0001:00000040       _NonMSIXInterruptHandler@8 00401040 f   rxdevice.obj
 0001:00000340       _PMCDpcResponseHandler@16  00401340 f   rxdevice.obj
 0001:000006f0       _PMCInterruptHandler@4     004016f0 f   rxdevice.obj
 0001:00000ae0       _PMCPushMessageUnitQueueFib@8 00401ae0 f   rxdevice.obj
 0001:00000dd0       _RxAccessDeviceRegister@8  00401dd0 f   rxdevice.obj
 0001:00000fe0       _RxCheckAdapterHealth@8    00401fe0 f   rxdevice.obj
 0001:00001080       _RxCheckSyncCommandComplete@8 00402080 f   rxdevice.obj
 0001:00001230       _RxDpcInterruptHandler@16  00402230 f   rxdevice.obj
 0001:00001240       _RxGetIBW@4                00402240 f   rxdevice.obj
 0001:00001270       _RxGetOMRx0@4              00402270 f   rxdevice.obj
 0001:000012c0       _RxInterruptHandler@4      004022c0 f   rxdevice.obj
 0001:00001500       _RxMapMailBoxFirmwareBase@4 00402500 f   rxdevice.obj
 0001:000015e0       _RxNewCommProcessInterrupt@8 004025e0 f   rxdevice.obj
 0001:00001990       _RxNotifyAdapter@12        00402990 f   rxdevice.obj
 0001:00001a40       _RxPullMessageUnitQueueCompletedFib@12 00402a40 f   rxdevice.obj
 0001:00001bf0       _RxPushMessageUnitQueueFib@8 00402bf0 f   rxdevice.obj
 0001:00001d20       _RxSendSynchCommand@48     00402d20 f   rxdevice.obj
 0001:000028f0       _RxStartAdapter@8          004038f0 f   rxdevice.obj
 0001:00002da0       _RxWaitForAdapterToBoot@4  00403da0 f   rxdevice.obj
 0001:00002ea0       _RxWriteIBW@8              00403ea0 f   rxdevice.obj
 0001:00002ef0       _RxWriteIDR@12             00403ef0 f   rxdevice.obj
 0001:00002f50       _RxWriteODR@12             00403f50 f   rxdevice.obj
 0001:00002fd0       _SetWaitCount4SendSyncCmd@8 00403fd0 f   rxdevice.obj
 0001:000030e0       _SetWaitCount4StartAdapter@4 004040e0 f   rxdevice.obj
 0001:00003150       _SimulateHbaFwTgtFailure@8 00404150 f   rxdevice.obj
 0001:00003210       _SimulateHbaScsiErros@8    00404210 f   rxdevice.obj
 0001:000032a0       _RevCheckCompatibility@12  004042a0 f   revision.obj
 0001:00003330       _RevGetBuildNumber@0       00404330 f   revision.obj
 0001:00003340       _RevGetExternalRev@0       00404340 f   revision.obj
 0001:00003350       _CompareStrings@12         00404350 f   helpers.obj
 0001:000033b0       _GetDriverParameter@20     004043b0 f   helpers.obj
 0001:000034b0       _LongToAscii@16            004044b0 f   helpers.obj
 0001:00003560       _MatchRegistryString@8     00404560 f   helpers.obj
 0001:00003610       _ZeroStructure@8           00404610 f   helpers.obj
 0001:00003630       _ArcPrintf                 00404630 f   arcdebug.obj
 0001:00003880       _ProcessCompleteSrbToHost@12 00404880 f   arcdebug.obj
 0001:000038b0       _PutItIntoInternalPrintBuffer@12 004048b0 f   arcdebug.obj
 0001:00003970       _RealSprintf@12            00404970 f   arcdebug.obj
 0001:00003dc0       _ChangeIoLimitAndPrintOutstanding@4 00404dc0 f   timer.obj
 0001:00003eb0       _CheckFWPulseInCrashDumpMode@4 00404eb0 f   timer.obj
 0001:00003fb0       _CheckingFWAfterPowerStateChange@4 00404fb0 f   timer.obj
 0001:00004410       _ConfigureContainersTimer@4 00405410 f   timer.obj
 0001:00004570       _DelayNotification@4       00405570 f   timer.obj
 0001:000045e0       _DequeueSortingQTimer@4    004055e0 f   timer.obj
 0001:000046b0       _MainTimeThread@4          004056b0 f   timer.obj
 0001:00004960       _RequestTimer@16           00405960 f   timer.obj
 0001:00004a00       _Reset_IOP_CompletionTimer@4 00405a00 f   timer.obj
 0001:00004f00       _RestartAdapterPendingTimer@4 00405f00 f   timer.obj
 0001:00004ff0       _ReturningKidnappedFibsToOS@4 00405ff0 f   timer.obj
 0001:00005090       _StopTimer@16              00406090 f   timer.obj
 0001:00005120       _SynchCommandCompletionTimer@4 00406120 f   timer.obj
 0001:000051d0       _SynchFibCompletionTimer@4 004061d0 f   timer.obj
 0001:000052c0       _UpdateThorHBAMappingTable@4 004062c0 f   timer.obj
 0001:000054f0       _VMCloseAllCompletionTimer@4 004064f0 f   timer.obj
 0001:00005700       _AllocateConsumerProducerCommArea@20 00406700 f   arcinit.obj
 0001:000059b0       _AllocateMessageUnitQueueCommArea@8 004069b0 f   arcinit.obj
 0001:00005e70       _ArcLogEventString@24      00406e70 f   arcinit.obj
 0001:00005f00       _AtomicINTXReleaseSlot@8   00406f00 f   arcinit.obj
 0001:00005f50       _CheckForVersionMisMatch@4 00406f50 f   arcinit.obj
 0001:00006080       _CheckMSIxPossibility@4    00407080 f   arcinit.obj
 0001:00006250       _ConfigureContainersRuntime@12 00407250 f   arcinit.obj
 0001:00006930       _DecToHex@4                00407930 f   arcinit.obj
 0001:000069a0       _DriverEntry@8             004079a0 f   arcinit.obj
 0001:00006a70       _DynamicallyThrottleLunQueueDepth@8 00407a70 f   arcinit.obj
 0001:00006cb0       _FindAdapter@24            00407cb0 f   arcinit.obj
 0001:00008960       _GetElapsedSeconds@4       00409960 f   arcinit.obj
 0001:000089f0       _GetFreeSlot@8             004099f0 f   arcinit.obj
 0001:00008a30       _GetThorHbaPhyDevInfo@4    00409a30 f   arcinit.obj
 0001:00008ee0       _HWSoftReset@4             00409ee0 f   arcinit.obj
 0001:000090c0       _HandleAdapterCommitConfig@4 0040a0c0 f   arcinit.obj
 0001:00009190       _HandleAdapterConfigIssues@4 0040a190 f   arcinit.obj
 0001:00009360       _HandleAdapterGetConfig@4  0040a360 f   arcinit.obj
 0001:00009470       _HwInitializeAdapter@4     0040a470 f   arcinit.obj
 0001:00009810       _ID_AllocateMem4CertainOBQ@12 0040a810 f   arcinit.obj
 0001:00009940       _ID_SetupMessageCap@8      0040a940 f   arcinit.obj
 0001:00009a30       _INTXGetFreeSlot@4         0040aa30 f   arcinit.obj
 0001:00009a60       _INTXReleaseSlot@8         0040aa60 f   arcinit.obj
 0001:00009aa0       _IOPReset@8                0040aaa0 f   arcinit.obj
 0001:00009f00       _InitializeConsumerProducerCommRegion@8 0040af00 f   arcinit.obj
 0001:0000a140       _InitializeConsumerProducerNewAdapter@12 0040b140 f   arcinit.obj
 0001:0000a200       _InitializeDPCs@4          0040b200 f   arcinit.obj
 0001:0000a690       _InitializeMessageUnitQueueNewAdapter@12 0040b690 f   arcinit.obj
 0001:0000a730       _IsAdapterReadyForConfigCommand@4 0040b730 f   arcinit.obj
 0001:0000a870       _LogSystemEvent@28         0040b870 f   arcinit.obj
 0001:0000a8d0       _MapDeviceBase@8           0040b8d0 f   arcinit.obj
 0001:0000ad50       _MatchPciIds@8             0040bd50 f   arcinit.obj
 0001:0000af40       _ReleaseSlot@12            0040bf40 f   arcinit.obj
 0001:0000af80       _ResetAdapter@8            0040bf80 f   arcinit.obj
 0001:0000b4e0       _ReturningLocalOutstandingRequestsToOS@4 0040c4e0 f   arcinit.obj
 0001:0000b5e0       _ReturningOutstandingSentToFWBeforeIOPResetToOS@4 0040c5e0 f   arcinit.obj
 0001:0000b6f0       _SA4ACI2Interface@4        0040c6f0 f   arcinit.obj
 0001:0000b7d0       _SA4CheckMSIx@4            0040c7d0 f   arcinit.obj
 0001:0000b820       _SA4OldCommInterface@4     0040c820 f   arcinit.obj
 0001:0000b860       _SA4StatusBatching@4       0040c860 f   arcinit.obj
 0001:0000b980       _SMCrashDumpModeInitAdapter@8 0040c980 f   arcinit.obj
 0001:0000bb90       _SMNormalModeInitAdapter@8 0040cb90 f   arcinit.obj
 0001:0000bf00       _SendEvent2OS@20           0040cf00 f   arcinit.obj
 0001:0000c6e0       _SendInitStructure@4       0040d6e0 f   arcinit.obj
 0001:0000ca00       _SetFwTime@4               0040da00 f   arcinit.obj
 0001:0000cd40       _CompleteQueuedRequest@12  0040dd40 f   cmddelivery.obj
 0001:0000ce20       _DequeueRawIoReadWriteRequest@12 0040de20 f   cmddelivery.obj
 0001:0000cfc0       _HandleInterrupt@4         0040dfc0 f   cmddelivery.obj
 0001:0000cfe0       _HandleMSIXInterrupt@8     0040dfe0 f   cmddelivery.obj
 0001:0000d0c0       _LocalDelay1us@0           0040e0c0 f   cmddelivery.obj
 0001:0000d0c0       _Delay1us@0                0040e0c0 f   arcdebug.obj
 0001:0000d120       _PollSmartHBAFIBCompletion@8 0040e120 f   cmddelivery.obj
 0001:0000d3c0       _PostProcessScsiCommand@16 0040e3c0 f   cmddelivery.obj
 0001:0000d6a0       _ProcessContainerInquiry@16 0040e6a0 f   cmddelivery.obj
 0001:0000dc90       _ProcessScsiCommand@12     0040ec90 f   cmddelivery.obj
 0001:0000e830       _QueuePrintf@12            0040f830 f   cmddelivery.obj
 0001:0000e8f0       _QueueRawIoReadWriteRequest@8 0040f8f0 f   cmddelivery.obj
 0001:0000f3b0       _SendFastIoFib@16          004103b0 f   cmddelivery.obj
 0001:0000f3e0       _SendFib@12                004103e0 f   cmddelivery.obj
 0001:0000f7c0       _SendRawIoFib@12           004107c0 f   cmddelivery.obj
 0001:0000faa0       _SendSynchFib@28           00410aa0 f   cmddelivery.obj
 0001:0000fc60       _StartIo@8                 00410c60 f   cmddelivery.obj
 0001:000105b0       _AdapterControl@12         004115b0 f   cmdproc.obj
 0001:00010ce0       _BuildHBAFib@12            00411ce0 f   cmdproc.obj
 0001:000111b0       _BuildHBAIoctlFib@20       004121b0 f   cmdproc.obj
 0001:00011420       _BuildIo@8                 00412420 f   cmdproc.obj
 0001:00011e40       _BuildRawIo2ScatterGather4HBAIoctl@16 00412e40 f   cmdproc.obj
 0001:00011fd0       _BuildRawIo2ScatterGather@12 00412fd0 f   cmdproc.obj
 0001:00012180       _BuildRawIoFib@12          00413180 f   cmdproc.obj
 0001:000124c0       _BuildRawIoScatterGather@12 004134c0 f   cmdproc.obj
 0001:00012680       _BuildReadWriteFib@12      00413680 f   cmdproc.obj
 0001:000129d0       _BuildScatterGather64@16   004139d0 f   cmdproc.obj
 0001:00012a80       _BuildScatterGather@16     00413a80 f   cmdproc.obj
 0001:00012b10       _BuildSrbFib@12            00413b10 f   cmdproc.obj
 0001:00012d80       _ConvertRawIo2ScatterGather@24 00413d80 f   cmdproc.obj
 0001:00012eb0       _InitializeFib@8           00413eb0 f   cmdproc.obj
 0001:00012ee0       _PrepareBMIC15@8           00413ee0 f   cmdproc.obj
 0001:00013120       _ReportFakeLuns@8          00414120 f   cmdproc.obj
 0001:00013170       _BuildRawScatterGather64@20 00414170 f   ioctl.obj
 0001:00013210       _BuildRawScatterGather@20  00414210 f   ioctl.obj
 0001:000132a0       _CSMIGetControllerConfig@8 004142a0 f   ioctl.obj
 0001:000133d0       _CSMIGetControllerStatus@8 004143d0 f   ioctl.obj
 0001:00013450       _CSMIGetDeviceAddress@8    00414450 f   ioctl.obj
 0001:000135a0       _CSMIGetDriverInfo@8       004145a0 f   ioctl.obj
 0001:00013620       _CSMIGetPhyInfo@8          00414620 f   ioctl.obj
 0001:00013780       _CSMIGetRAIDConfig@8       00414780 f   ioctl.obj
 0001:000139a0       _CSMIGetRAIDInfo@8         004149a0 f   ioctl.obj
 0001:00013af0       _CSMIGetSATASignature@8    00414af0 f   ioctl.obj
 0001:00013c50       _CSMIGetSCSIAddress@8      00414c50 f   ioctl.obj
 0001:00013da0       _CSMISTPPassThru@8         00414da0 f   ioctl.obj
 0001:00013fd0       _HandleCSMI@8              00414fd0 f   ioctl.obj
 0001:000140c0       _ProcessIoctl@12           004150c0 f   ioctl.obj
 0001:00016590       _AdapterIsAlive@4          00417590 f   comm.obj
 0001:000165d0       _CompleteAllSortingQueue@8 004175d0 f   comm.obj
 0001:00016650       _CompleteBufferedRequest@12 00417650 f   comm.obj
 0001:00016700       _CompleteSortingQueueRequest@12 00417700 f   comm.obj
 0001:00016790       _DeQueueSortingQueue@8     00417790 f   comm.obj
 0001:00016930       _DpcDequeueRawIoReadWriteRequest@16 00417930 f   comm.obj
 0001:000169a0       _FreeConsumerProducerAif@8 004179a0 f   comm.obj
 0001:00016a80       _GetConsumerProducerCompletedFib@12 00417a80 f   comm.obj
 0001:00016b20       _GetMessageUnitQueueCompletedFib@12 00417b20 f   comm.obj
 0001:00016b40       _GetQueueEntry@16          00417b40 f   comm.obj
 0001:00016c90       _ProcessAif@8              00417c90 f   comm.obj
 0001:00016fb0       _ProcessHbaErrors@12       00417fb0 f   comm.obj
 0001:00017400       _ProcessNormalFib@20       00418400 f   comm.obj
 0001:00017e00       _QueueSortingQ@8           00418e00 f   comm.obj
 0001:00018070       _RestoreBMIC15Srb@8        00419070 f   comm.obj
 0001:00018140       _SendConsumerProducerFib@4 00419140 f   comm.obj
 0001:000181b0       _SendMessageUnitQueueFib@4 004191b0 f   comm.obj
 0001:00018240       _ServiceHostCommandNormalQueue@4 00419240 f   comm.obj
 0001:000182e0       _ServiceHostResponseNormalQueue@4 004192e0 f   comm.obj
 0001:00018680       _ServiceInternalAifQueue@4 00419680 f   comm.obj
 0001:00018720       _SubDeQueueSortingQueue@8  00419720 f   comm.obj
 0001:000187f0       _HwScsiWmiExecuteMethod@32 004197f0 f   wmi.obj
 0001:00018890       _HwScsiWmiFunctionControl@20 00419890 f   wmi.obj
 0001:000188b0       _HwScsiWmiQueryDataBlock@32 004198b0 f   wmi.obj
 0001:000188d0       _HwScsiWmiQueryReginfo@12  004198d0 f   wmi.obj
 0001:000188f0       _HwScsiWmiSetDataBlock@24  004198f0 f   wmi.obj
 0001:00018900       _HwScsiWmiSetDataItem@28   00419900 f   wmi.obj
 0001:00018910       _InitializeWmiInterface@4  00419910 f   wmi.obj
 0001:00018a10       _ProcessWmi@8              00419a10 f   wmi.obj
 0001:00018a70       _GsDriverEntry@8           00419a70 f   BufferOverflowFastFailK:gs_driverentry.obj
 0001:00018a86       @__security_check_cookie@4 00419a86 f   BufferOverflowFastFailK:secchk.obj
 0001:00018a9c       ___report_gsfailure        00419a9c f   BufferOverflowFastFailK:gs_report.obj
 0001:00018ab0       ___report_rangecheckfailure 00419ab0 f   BufferOverflowFastFailK:gs_report.obj
 0001:00018aba       _memset                    00419aba f   ntoskrnl:ntoskrnl.exe
 0001:00018ac6       __aulldvrm                 00419ac6 f   ntoskrnl:ntoskrnl.exe
 0001:00018ad2       _ExSystemTimeToLocalTime@8 00419ad2 f   ntoskrnl:ntoskrnl.exe
 0001:00018ade       _RtlTimeToTimeFields@8     00419ade f   ntoskrnl:ntoskrnl.exe
 0001:00018aea       __alldiv                   00419aea f   ntoskrnl:ntoskrnl.exe
 0001:00018af6       __allmul                   00419af6 f   ntoskrnl:ntoskrnl.exe
 0001:00018b02       __aulldiv                  00419b02 f   ntoskrnl:ntoskrnl.exe
 0001:00018b0e       __aullshr                  00419b0e f   ntoskrnl:ntoskrnl.exe
 0001:00018b1a       _ScsiPortWmiDispatchFunction@28 00419b1a f   scsiwmi:wmilib.obj
 0001:00018b96       _ScsiWmipProcessRequest@36 00419b96 f   scsiwmi:wmilib.obj
 0001:00018f18       _ScsiPortWmiPostProcess@12 00419f18 f   scsiwmi:wmilib.obj
 0001:00018f48       _ScsiWmipPostProcess@24    00419f48 f   scsiwmi:wmilib.obj
 0001:000190b2       _ScsiWmipFindGuid@20       0041a0b2 f   scsiwmi:wmilib.obj
 0001:00019102       _ULongAdd@12               0041a102 f i scsiwmi:wmilib.obj
 0001:00019130       _ForceSEHExceptionHandler@16 0041a130 f   BufferOverflowFastFailK:forceseh.obj
 0001:00019138       ??_C@_0CJ@KAGJNHLI@OMR?5value?5in?5Check?5Adapter?5Healt@FNODOBFM@ 0041a138     rxdevice.obj
 0001:00019162       ??_C@_0DE@IHDJGLJF@This?5should?5not?5happen?4?5We?5only?5@FNODOBFM@ 0041a162     rxdevice.obj
 0001:00019196       ??_C@_0CP@PEAJGKJE@?$CK?5NonMSIXInterruptHandle?3?5pFibCo@FNODOBFM@ 0041a196     rxdevice.obj
 0001:000191c6       ??_C@_0EM@CCDNION@?$CK?5Start?5a?5timer?5to?5update?5contai@FNODOBFM@ 0041a1c6     rxdevice.obj
 0001:00019212       ??_C@_0DL@DMOOFJIN@?$CK?53?124?3?5pFibContext?$DNNULL?5?$CB?$CBline?5@FNODOBFM@ 0041a212     rxdevice.obj
 0001:0001924e       ??_C@_0ED@DAJFCMJP@?$CK?5Start?5a?5timer?5to?5update?5Contai@FNODOBFM@ 0041a24e     rxdevice.obj
 0001:00019292       ??_C@_0BF@JNCAAJNE@pFibContext?$DNNULL?5?$CB?$CB?6?$AA@FNODOBFM@ 0041a292     rxdevice.obj
 0001:000192a8       ??_C@_0EI@DKKBIMEF@?$CK?5Start?5a?5timer?5to?5update?5contai@FNODOBFM@ 0041a2a8     rxdevice.obj
 0001:000192f0       ??_C@_0FE@JLKFMCPA@?$CK?5PMCPushMessageUnitQueueFib?3?5Cm@FNODOBFM@ 0041a2f0     rxdevice.obj
 0001:00019344       ??_C@_0FE@JICOMBJP@?$CK?5PMCPushMessageUnitQueueFib?3?5Cm@FNODOBFM@ 0041a344     rxdevice.obj
 0001:00019398       ??_C@_0HN@JEPKAECC@?$CK?5RxSendSynchCommand?3?5Thor?5AIF?5e@FNODOBFM@ 0041a398     rxdevice.obj
 0001:00019416       ??_C@_0EC@LAPIEKPJ@?$CK?5RxSendSynchCommand?3?5mailbox?$FL0?$FN@FNODOBFM@ 0041a416     rxdevice.obj
 0001:00019458       ??_C@_0DJ@GJNDHOED@?$CK?5RxSendSynchCommand?3?5mailbox?$FL0?$FN@FNODOBFM@ 0041a458     rxdevice.obj
 0001:00019492       ??_C@_0HK@NJDHDGMI@?$CK?5RxSendSynchCommand?3?5There?5is?5a@FNODOBFM@ 0041a492     rxdevice.obj
 0001:0001950c       ??_C@_0HB@PLCHFMAA@?$CK?5RxSendSynchCommand?3?5synch?5cmd?3@FNODOBFM@ 0041a50c     rxdevice.obj
 0001:0001957e       ??_C@_0FD@ECFFGBJE@?5RxSendSynchCommand?3?5FW?5doing?5IO@FNODOBFM@ 0041a57e     rxdevice.obj
 0001:000195d2       ??_C@_0FE@DOFCONDK@?$CK?5RxSendSynchCommand?3?5wait?5for?5F@FNODOBFM@ 0041a5d2     rxdevice.obj
 0001:00019626       ??_C@_0GF@LFEFAJKJ@?5RxSendSynchCommand?5?$CIcrash?5dump?5@FNODOBFM@ 0041a626     rxdevice.obj
 0001:0001968c       ??_C@_0GF@CDCMENMG@?$CK?5RxSendSynchCommand?5?$CIcrash?5dump@FNODOBFM@ 0041a68c     rxdevice.obj
 0001:000196f2       ??_C@_0EL@HOIBIGPI@?$CK?5RxSendSynchCommand?3?5Got?5respon@FNODOBFM@ 0041a6f2     rxdevice.obj
 0001:0001973e       ??_C@_0EJ@DGPABBLG@?$CK?5RxSendSynchCommand?3?5Should?5NOT@FNODOBFM@ 0041a73e     rxdevice.obj
 0001:00019788       ??_C@_0FA@HKIBFKMH@?$CK?5RxSendSynchCommand?3?5Still?5NO?5r@FNODOBFM@ 0041a788     rxdevice.obj
 0001:000197d8       ??_C@_0KI@HMCHOJIN@?5RxSendSynchCommand?$FLMSIX?5mode?$FN?5f@FNODOBFM@ 0041a7d8     rxdevice.obj
 0001:00019880       ??_C@_0JP@JKCHEOCJ@?5RxSendSynchCommand?$FLMSIX?5mode?$FN?3?5@FNODOBFM@ 0041a880     rxdevice.obj
 0001:00019920       ??_C@_0CN@BCCBJMEA@?5RxSendSynchCommand?5Failed?5?$CFd?0wa@FNODOBFM@ 0041a920     rxdevice.obj
 0001:0001994e       ??_C@_0DB@JEAHJGPL@?$CK?5pDeviceExtension?9?$DOMaxMSIXVecto@FNODOBFM@ 0041a94e     rxdevice.obj
 0001:00019980       ??_C@_0CB@JPABDNKH@?$CK?5Begins?5StatusBatching?0?5Yeaaa?$CB?6@FNODOBFM@ 0041a980     rxdevice.obj
 0001:000199a2       ??_C@_0CF@BPKEMKA@?$CK?5ACI2?5Command?5Delivery?5is?5enabl@FNODOBFM@ 0041a9a2     rxdevice.obj
 0001:000199c8       ??_C@_1DK@JBHFOPMP@?$AAA?$AAd?$AAa?$AAp?$AAt?$AAe?$AAr?$AA?5?$AAC?$AAo?$AAn?$AAf?$AAi?$AAg?$AAu?$AAr?$AAa?$AAt?$AAi?$AAo?$AAn?$AA?5?$AAf?$AAa?$AAi?$AAl?$AAe?$AAd?$AA?$AA@FNODOBFM@ 0041a9c8     rxdevice.obj
 0001:00019a02       ??_C@_02DKCKIIND@?$CFs?$AA@FNODOBFM@ 0041aa02     arcdebug.obj
 0001:00019a06       ??_C@_06NBLAGFFP@Archba?$AA@FNODOBFM@ 0041aa06     arcdebug.obj
 0001:00019a0e       ??_C@_0BC@JKBDDNDF@DelayNotification?$AA@FNODOBFM@ 0041aa0e     timer.obj
 0001:00019a20       ??_C@_0CK@BKKGBKDP@?$CK?5Scan?5Notification?5sent?5in?5?$CFs?5?$CI@FNODOBFM@ 0041aa20     timer.obj
 0001:00019a4a       ??_C@_0GB@FAGGLJPH@?$CK?5First?58?5HBA?5devices?3?5?$CI0x?$CFx?0?$CFd?$CJ@FNODOBFM@ 0041aa4a     timer.obj
 0001:00019aac       ??_C@_0FN@EKAEFPGA@?$CK?5HBA?5mapping?5table?5updated?0?5tim@FNODOBFM@ 0041aaac     timer.obj
 0001:00019b0a       ??_C@_0GF@PMGNJLIM@?$CK?5Start?5a?5timer?5to?5update?5Contai@FNODOBFM@ 0041ab0a     timer.obj
 0001:00019b70       ??_C@_0CK@JLKEFPAM@entering?5CheckingFWAfterPowerSta@FNODOBFM@ 0041ab70     timer.obj
 0001:00019b9a       ??_C@_0GN@GHJFFNOA@?$CK?5set?5timer?5AGAIN?5in?5CheckingFWA@FNODOBFM@ 0041ab9a     timer.obj
 0001:00019c08       ??_C@_0FK@MIIMDOAD@?$CK?5set?5timer?5AGAIN?5in?5CheckingFWA@FNODOBFM@ 0041ac08     timer.obj
 0001:00019c62       ??_C@_0GB@EDFGCDFC@?$CK?5set?5timer?5AGAIN?5in?5CheckingFWA@FNODOBFM@ 0041ac62     timer.obj
 0001:00019cc4       ??_C@_0N@JEADMAEG@7?45?40?450666?$AA?$AA@FNODOBFM@ 0041acc4     timer.obj
 0001:00019cd2       ??_C@_0DO@GCDGNMH@?$CK?5FW?5is?5back?5from?5S3?1S4?4?5StorPor@FNODOBFM@ 0041acd2     timer.obj
 0001:00019d10       ??_C@_0DM@JABFAEPO@?$CK?5?9?5Reset?5AIFSrb?5to?5NULL?5when?5ba@FNODOBFM@ 0041ad10     timer.obj
 0001:00019d4c       ??_C@_0DN@ELHOMNDM@?$CK?5leaving?5CheckingFWAfterPowerSt@FNODOBFM@ 0041ad4c     timer.obj
 0001:00019d8a       ??_C@_0DO@OBELKDEH@?$CK?5set?5timer?5AGAIN?5to?5check?5the?5F@FNODOBFM@ 0041ad8a     timer.obj
 0001:00019dc8       ??_C@_0CI@JPJEKICG@DPC?9Timeout?5may?5happen?5in?5ResetA@FNODOBFM@ 0041adc8     timer.obj
 0001:00019df0       ??_C@_0DH@JNGKJDAE@One?5kidnapped?5FIB?5released?$CB?5FIB_@FNODOBFM@ 0041adf0     timer.obj
 0001:00019e28       ??_C@_0EJ@PCDGPKJP@?$CK?5Driver?5was?5not?5able?5to?5send?5?$CFd@FNODOBFM@ 0041ae28     timer.obj
 0001:00019e72       ??_C@_0DM@PNDEAHOI@?$CK?5Send?5BusChangeDetected?5to?5OS?5i@FNODOBFM@ 0041ae72     timer.obj
 0001:00019eae       ??_C@_0EH@FCLGCKBJ@?$CK?5Start?5a?5timer?5to?5update?5HBA?5de@FNODOBFM@ 0041aeae     timer.obj
 0001:00019ef6       ??_C@_0GE@IFJDDHGE@?$CK?5Start?5a?5timer?5to?5update?5Contai@FNODOBFM@ 0041aef6     timer.obj
 0001:00019f5a       ??_C@_0DL@DODBJONE@?$CK?5SynchCommandCompletionTimer?3?5S@FNODOBFM@ 0041af5a     timer.obj
 0001:00019f96       ??_C@_0EO@CBNEAKKI@?$CK?5VMCloseAllCompletionTimer?3?5sen@FNODOBFM@ 0041af96     timer.obj
 0001:00019fe4       ??_C@_0FI@MJCPBEAD@?$CK?5VMCloseAllCompletionTimer?3?5wai@FNODOBFM@ 0041afe4     timer.obj
 0001:0001a03c       ??_C@_0DO@ELMMCKMD@?$CK?5VMCloseAllCompletionTimer?3?5SRB@FNODOBFM@ 0041b03c     timer.obj
 0001:0001a07a       ??_C@_0EH@BGEEAOIJ@?$CK?5VMCloseAllCompletionTimer?3?5Sho@FNODOBFM@ 0041b07a     timer.obj
 0001:0001a0c2       ??_C@_0EF@HLMPMNBN@?$CK?5VMCloseAllCompletionTimer?3?5Syn@FNODOBFM@ 0041b0c2     timer.obj
 0001:0001a108       ??_C@_0DH@IBACIAED@?$CK?5SynchFibCompletionTimer?3?5SyncF@FNODOBFM@ 0041b108     timer.obj
 0001:0001a140       ??_C@_0DP@OKLOLMOG@?5IBW_SWR?5register?5value?50?0?5reset@FNODOBFM@ 0041b140     timer.obj
 0001:0001a180       ??_C@_0FK@ODMKKBJL@?$CK?5Start?5a?5timer?5to?5update?5Contai@FNODOBFM@ 0041b180     timer.obj
 0001:0001a1da       ??_C@_0FH@GFIHLMMH@?$CK?5Start?5a?5timer?5to?5update?5Contai@FNODOBFM@ 0041b1da     timer.obj
 0001:0001a232       ??_C@_0DH@KAAGAFOD@?$CK?5leaving?5Reset_IOP_CompletionTi@FNODOBFM@ 0041b232     timer.obj
 0001:0001a26a       ??_C@_0CD@MKPFBJDC@leaving?5Reset_IOP_CompletionTime@FNODOBFM@ 0041b26a     timer.obj
 0001:0001a28e       ??_C@_0DL@DOEFCINE@?$CK?5HW?5SOFT?5RESET?5done?4?5StorPort?5m@FNODOBFM@ 0041b28e     timer.obj
 0001:0001a2ca       ??_C@_0DH@DFJOPAAJ@?$CK?5RESET?5IOP?5done?4?5StorPort?5minip@FNODOBFM@ 0041b2ca     timer.obj
 0001:0001a302       ??_C@_0CK@OJIMCPJO@Kernel?5Panic?5BlinkLed?5Code?5?$CFx?5?0?5@FNODOBFM@ 0041b302     timer.obj
 0001:0001a32c       ??_C@_0CL@KFLNLOFE@IOP_HWSOFT_RESET?3?5FW?5status?5?$CFx?5?0@FNODOBFM@ 0041b32c     timer.obj
 0001:0001a358       ??_C@_0EF@BBNOBECH@?$CK?5set?5timer?5AGAIN?5to?5check?5the?5F@FNODOBFM@ 0041b358     timer.obj
 0001:0001a39e       ??_C@_0EC@MICIKMJM@?$CK?5set?5timer?5AGAIN?5to?5check?5the?5F@FNODOBFM@ 0041b39e     timer.obj
 0001:0001a3e0       ??_C@_0BJ@HIBCALL@ProcessAgeOfSortingQueue?$AA@FNODOBFM@ 0041b3e0     timer.obj
 0001:0001a3fa       ??_C@_0DA@GEMOEFPE@Dequeue?5Sorting?5Queue?5failed?5in?5@FNODOBFM@ 0041b3fa     timer.obj
 0001:0001a42a       ??_C@_0ID@HFHPGANL@Dequeue?5Sorting?5Queue?5failed?5whe@FNODOBFM@ 0041b42a     timer.obj
 0001:0001a4ae       ??_C@_0CL@MJMGCLDD@entering?5AllocateConsumerProduce@FNODOBFM@ 0041b4ae     arcinit.obj
 0001:0001a4da       ??_C@_0DK@IJIOFPFH@leaving?5AllocateConsumerProducer@FNODOBFM@ 0041b4da     arcinit.obj
 0001:0001a514       ??_C@_0CI@FFOEPFMJ@?$CK?5ConsumerProducerCommArea?0?5VAdd@FNODOBFM@ 0041b514     arcinit.obj
 0001:0001a53c       ??_C@_0CN@MBHLABKL@?$CK?5Adapter?5got?5an?5invalid?5host?5me@FNODOBFM@ 0041b53c     arcinit.obj
 0001:0001a56a       ??_C@_0DJ@JGKEIEFI@leaving?5AllocateConsumerProducer@FNODOBFM@ 0041b56a     arcinit.obj
 0001:0001a5a4       ??_C@_0CL@KCDMGIOM@entering?5AllocateMessageUnitQueu@FNODOBFM@ 0041b5a4     arcinit.obj
 0001:0001a5d0       ??_C@_0FP@JFBPKCDF@?$CK?5AllocateMessageUnitQueueCommAr@FNODOBFM@ 0041b5d0     arcinit.obj
 0001:0001a630       ??_C@_0DM@JMMHKBOC@?$CK?5AllocateMessageUnitQueueCommAr@FNODOBFM@ 0041b630     arcinit.obj
 0001:0001a66c       ??_C@_0DK@BKFHOPDI@leaving?5AllocateMessageUnitQueue@FNODOBFM@ 0041b66c     arcinit.obj
 0001:0001a6a6       ??_C@_0DA@ICFHAOHF@?$CK?5AllocateMessageUnitQueueCommAr@FNODOBFM@ 0041b6a6     arcinit.obj
 0001:0001a6d6       ??_C@_0FB@FDJPGKAF@?$CK?5StorPortAllocateContiguousMemo@FNODOBFM@ 0041b6d6     arcinit.obj
 0001:0001a728       ??_C@_0FB@MMEFOJJL@?$CK?5StorPortAllocateContiguousMemo@FNODOBFM@ 0041b728     arcinit.obj
 0001:0001a77a       ??_C@_0BJ@OICKMJHC@?$CK?5pBuf1?$DN0x?$CFp?0pBuf2?$DN0x?$CFp?6?$AA@FNODOBFM@ 0041b77a     arcinit.obj
 0001:0001a794       ??_C@_0BO@DPONBFMO@?$CK?5MemoryPhysicalAddress?$DN0x?$CFp?6?$AA@FNODOBFM@ 0041b794     arcinit.obj
 0001:0001a7b2       ??_C@_0EL@ELLGMDMB@?$CK?5Allocate?5big?5IOCTL?5buffer?5succ@FNODOBFM@ 0041b7b2     arcinit.obj
 0001:0001a7fe       ??_C@_0DJ@EGOLHGNF@leaving?5AllocateMessageUnitQueue@FNODOBFM@ 0041b7fe     arcinit.obj
 0001:0001a838       ??_C@_0CF@DNFJFJLG@entering?5ConfigureContainersRunt@FNODOBFM@ 0041b838     arcinit.obj
 0001:0001a85e       ??_C@_0EJ@GFICDCBB@?$CK?5ConfigureContainersRuntime?3?5Re@FNODOBFM@ 0041b85e     arcinit.obj
 0001:0001a8a8       ??_C@_0EF@KJEEMCEN@?$CK?5ConfigureContainersRuntime?3?5Ge@FNODOBFM@ 0041b8a8     arcinit.obj
 0001:0001a8ee       ??_C@_0EF@JADMGPAN@?$CK?5ConfigureContainersRuntime?3?5Ge@FNODOBFM@ 0041b8ee     arcinit.obj
 0001:0001a934       ??_C@_0EM@NKPEDKJ@?$CK?5ConfigureContainersRuntime?3?5no@FNODOBFM@ 0041b934     arcinit.obj
 0001:0001a980       ??_C@_0EF@ECHMIPBP@?$CK?5Found?5a?5new?5container?5?9?5tid?3?5?$CF@FNODOBFM@ 0041b980     arcinit.obj
 0001:0001a9c6       ??_C@_0DK@FCJKMAGD@ConfigureContainersRuntime?3?5UID?5@FNODOBFM@ 0041b9c6     arcinit.obj
 0001:0001aa00       ??_C@_0DK@PHPDGAOG@?$CK?5ConfigureContainersRuntime?3?5di@FNODOBFM@ 0041ba00     arcinit.obj
 0001:0001aa3a       ??_C@_0GG@BFFFADFC@?$CK?5ConfigureContainersRuntime?3?5Fa@FNODOBFM@ 0041ba3a     arcinit.obj
 0001:0001aaa0       ??_C@_0EA@JBBLNOGE@?$CK?5ConfigureContainersRuntime?3?5RA@FNODOBFM@ 0041baa0     arcinit.obj
 0001:0001aae0       ??_C@_0EB@GBLPFGID@?$CK?5ConfigureContainersRuntime?3?5Di@FNODOBFM@ 0041bae0     arcinit.obj
 0001:0001ab22       ??_C@_0CO@FOBCLEMJ@?$CK?5ConfigureContainersRuntime?3?5di@FNODOBFM@ 0041bb22     arcinit.obj
 0001:0001ab50       ??_C@_0DO@KMBICFHC@?$CK?5ConfigureContainersRuntime?3?5Sy@FNODOBFM@ 0041bb50     arcinit.obj
 0001:0001ab8e       ??_C@_0DB@JMFIFBDA@leaving?5ConfigureContainersRunti@FNODOBFM@ 0041bb8e     arcinit.obj
 0001:0001abc0       ??_C@_0CC@KOGKIGDL@entering?5CheckForVersionMisMatch@FNODOBFM@ 0041bbc0     arcinit.obj
 0001:0001abe2       ??_C@_0CB@BOFDNAKM@This?5is?5a?5code?5stream?5identifier@FNODOBFM@ 0041bbe2     arcinit.obj
 0001:0001ac04       ??_C@_1CE@PCDJGPON@?$AAB?$AAa?$AAd?$AA?5?$AAV?$AAe?$AAr?$AAs?$AAi?$AAo?$AAn?$AA?5?$AAM?$AAa?$AAt?$AAc?$AAh?$AA?$AA@FNODOBFM@ 0041bc04     arcinit.obj
 0001:0001ac28       ??_C@_0DF@MNNMPGOO@?$CK?5Version?5Mismatch?3?5Bios?3?$CFd?0?5Fir@FNODOBFM@ 0041bc28     arcinit.obj
 0001:0001ac5e       ??_C@_0EC@DEDLMEPI@leving?5CheckForVersionMisMatch?5w@FNODOBFM@ 0041bc5e     arcinit.obj
 0001:0001aca0       ??_C@_0BN@GKEKJNDP@?$CFs?5Driver?5entry?5rtnval?5?$DN?5?$CFx?6?$AA@FNODOBFM@ 0041bca0     arcinit.obj
 0001:0001acbe       ??_C@_0DD@FIIKPLIC@?$CFs?3?5Driver?5FindAdapter?5?9?5invalid@FNODOBFM@ 0041bcbe     arcinit.obj
 0001:0001acf2       ??_C@_0M@NCHBOPE@kernalprint?$AA@FNODOBFM@ 0041bcf2     arcinit.obj
 0001:0001acfe       ??_C@_0BE@IDLOJBGB@?$CK?5KERNAL?5PRINT?5?$DN?51?6?$AA@FNODOBFM@ 0041bcfe     arcinit.obj
 0001:0001ad12       ??_C@_0BG@INJAEJHE@entering?5FindAdapter?6?$AA@FNODOBFM@ 0041bd12     arcinit.obj
 0001:0001ad28       ??_C@_0FD@NLKPIIHJ@?$CK?5This?5is?5WS03?5R2?0?5Vista?5or?5Long@FNODOBFM@ 0041bd28     arcinit.obj
 0001:0001ad7c       ??_C@_0FF@EIPBDAPC@?$CK?$CK?$CK?$CK?$CK?5Size?5of?5PORT_CONFIGURATION@FNODOBFM@ 0041bd7c     arcinit.obj
 0001:0001add2       ??_C@_0EF@MDPAOPOH@?$CK?5HwScsiFindAdapter?3?5DeviceExten@FNODOBFM@ 0041bdd2     arcinit.obj
 0001:0001ae18       ??_C@_0CD@BBBDOKPE@?$CK?5Returned?5PCI?5bus?5data?5length?$DN?$CF@FNODOBFM@ 0041be18     arcinit.obj
 0001:0001ae3c       ??_C@_0BB@ELNGMCEN@BreakPointHelper?$AA@FNODOBFM@ 0041be3c     arcinit.obj
 0001:0001ae4e       ??_C@_0BN@NMODDHNP@?$CK?53?5seconds?5waiting?5is?5done?6?$AA@FNODOBFM@ 0041be4e     arcinit.obj
 0001:0001ae6c       ??_C@_0DD@OAOECDIB@leaving?5FindAdapter?5?9?5StorPortGe@FNODOBFM@ 0041be6c     arcinit.obj
 0001:0001aea0       ??_C@_0DF@ODNFGMFG@?$CK?5leaving?5FindAdapter?5?9?5StorPort@FNODOBFM@ 0041bea0     arcinit.obj
 0001:0001aed6       ??_C@_0BN@FJDEMAMC@?$CK?50x40?5PCI?5Bus?5Data?5read?5in?6?$AA@FNODOBFM@ 0041bed6     arcinit.obj
 0001:0001aef4       ??_C@_0BN@INBKDNHG@?$CK?50xFF?5PCI?5Bus?5Data?5read?5in?6?$AA@FNODOBFM@ 0041bef4     arcinit.obj
 0001:0001af12       ??_C@_0DB@DAIGEFPJ@?$CK?5No?5Support?5on?5Capabilties?5list@FNODOBFM@ 0041bf12     arcinit.obj
 0001:0001af44       ??_C@_0BM@KCLFMKNE@?$CK?5Capability_offset?5?$DN?50x?$CFx?5?$AA@FNODOBFM@ 0041bf44     arcinit.obj
 0001:0001af60       ??_C@_0BJ@KNABCMMM@?5?9?9?$DOcapabilty_id?5?$DN?50x?$CFx?6?$AA@FNODOBFM@ 0041bf60     arcinit.obj
 0001:0001af7a       ??_C@_0BK@JIIOJNIO@?$CK?5Message_control?5?$DN?50x?$CFx?6?$AA@FNODOBFM@ 0041bf7a     arcinit.obj
 0001:0001af94       ??_C@_0BF@HNFCBKLM@?$CK?5HW?5supports?5MSI?9X?6?$AA@FNODOBFM@ 0041bf94     arcinit.obj
 0001:0001afaa       ??_C@_0L@BLEMHNKF@archbamode?$AA@FNODOBFM@ 0041bfaa     arcinit.obj
 0001:0001afb6       ??_C@_0BM@OFPMAGCK@?$CK?5ARC?5HBA?5MODE?5setting?3?5?$CFd?6?$AA@FNODOBFM@ 0041bfb6     arcinit.obj
 0001:0001afd2       ??_C@_09LEIBFFMJ@forceintx?$AA@FNODOBFM@ 0041bfd2     arcinit.obj
 0001:0001afdc       ??_C@_0N@FCLAIEBP@forcepolling?$AA@FNODOBFM@ 0041bfdc     arcinit.obj
 0001:0001afea       ??_C@_0DI@MNEPEDIK@?$CK?5StorPortGetActiveGroupCount?5ha@FNODOBFM@ 0041bfea     arcinit.obj
 0001:0001b022       ??_C@_0ED@JJDFFHPI@?$CK?5StorPortGetActiveGroupCount?5re@FNODOBFM@ 0041c022     arcinit.obj
 0001:0001b066       ??_C@_0DJ@FDFDEBND@?$CK?5StorPortGetHighestNodeNumber?5h@FNODOBFM@ 0041c066     arcinit.obj
 0001:0001b0a0       ??_C@_0EL@PIGODLHL@?$CK?5StorPortGetHighestNodeNumber?5r@FNODOBFM@ 0041c0a0     arcinit.obj
 0001:0001b0ec       ??_C@_0EM@HBPALBEJ@?$CK?5StorPortGetHighestNodeNumber?5r@FNODOBFM@ 0041c0ec     arcinit.obj
 0001:0001b138       ??_C@_0DF@EDOFIEGL@?$CK?5StorPortGetGroupAffinity?5has?5n@FNODOBFM@ 0041c138     arcinit.obj
 0001:0001b16e       ??_C@_0HE@CADMEBCK@?$CK?5StorPortGetGroupAffinity?5retur@FNODOBFM@ 0041c16e     arcinit.obj
 0001:0001b1e2       ??_C@_0EI@OFPHCHHN@?$CK?5StorPortGetGroupAffinity?5retur@FNODOBFM@ 0041c1e2     arcinit.obj
 0001:0001b22a       ??_C@_0EO@MADFJJKE@?$CK?5StorPortGetGroupAffinity?5retur@FNODOBFM@ 0041c22a     arcinit.obj
 0001:0001b278       ??_C@_0P@JECJMKHH@runspecialcode?$AA@FNODOBFM@ 0041c278     arcinit.obj
 0001:0001b288       ??_C@_0BI@LHEEIHDL@?$CK?5RUN?5SPECIAL?5CODE?5?$DN?51?6?$AA@FNODOBFM@ 0041c288     arcinit.obj
 0001:0001b2a0       ??_C@_0BI@LGIGONAM@?$CK?5RUN?5SPECIAL?5CODE?5?$DN?50?6?$AA@FNODOBFM@ 0041c2a0     arcinit.obj
 0001:0001b2b8       ??_C@_0M@KNIKEID@kidnapvalve?$AA@FNODOBFM@ 0041c2b8     arcinit.obj
 0001:0001b2c4       ??_C@_0BF@CEDJMGLL@?$CK?5KIDNAP?5VALVE?5?$DN?5?$CFd?6?$AA@FNODOBFM@ 0041c2c4     arcinit.obj
 0001:0001b2da       ??_C@_0O@OCGMBHKL@checkinterval?$AA@FNODOBFM@ 0041c2da     arcinit.obj
 0001:0001b2e8       ??_C@_0CM@FEFEBKKC@?$CK?5IOP?5RESET?5COMPLETION?5Check?5Int@FNODOBFM@ 0041c2e8     arcinit.obj
 0001:0001b314       ??_C@_0N@MOEJGNKK@stallseconds?$AA@FNODOBFM@ 0041c314     arcinit.obj
 0001:0001b322       ??_C@_0BG@DLFLFJEO@?$CK?5STALL?5SECONDS?5?$DN?5?$CFd?6?$AA@FNODOBFM@ 0041c322     arcinit.obj
 0001:0001b338       ??_C@_0O@BPMKJHCJ@hbaqueuedepth?$AA@FNODOBFM@ 0041c338     arcinit.obj
 0001:0001b346       ??_C@_0BI@IIHNBKPK@?$CK?5HBA?5QUEUE?5DEPTH?5?$DN?5?$CFd?6?$AA@FNODOBFM@ 0041c346     arcinit.obj
 0001:0001b35e       ??_C@_04GGLOKIEE@dump?$AA@FNODOBFM@ 0041c35e     arcinit.obj
 0001:0001b364       ??_C@_05FDLGEGEK@ntldr?$AA@FNODOBFM@ 0041c364     arcinit.obj
 0001:0001b36a       ??_C@_05PMICOLGA@hiber?$AA@FNODOBFM@ 0041c36a     arcinit.obj
 0001:0001b370       ??_C@_0CD@JEMNEMMP@?$CK?$CK?$CK?$CK?5dump?5?$HM?5ntldr?5?$HM?5hiber?5is?5TRU@FNODOBFM@ 0041c370     arcinit.obj
 0001:0001b394       ??_C@_0BK@NELCFLHO@?$CK?5Switching?5to?5INTx?5mode?6?$AA@FNODOBFM@ 0041c394     arcinit.obj
 0001:0001b3ae       ??_C@_09IPELKJIO@BLEDCheck?$AA@FNODOBFM@ 0041c3ae     arcinit.obj
 0001:0001b3b8       ??_C@_0L@NIPCGJOG@DPCAllowed?$AA@FNODOBFM@ 0041c3b8     arcinit.obj
 0001:0001b3c4       ??_C@_09CHINNNMJ@CSMI?$DNNone?$AA@FNODOBFM@ 0041c3c4     arcinit.obj
 0001:0001b3ce       ??_C@_0BA@BKKNJKOP@CSMI?$DNRestricted?$AA@FNODOBFM@ 0041c3ce     arcinit.obj
 0001:0001b3de       ??_C@_09PKBPEONE@CSMI?$DNFull?$AA@FNODOBFM@ 0041c3de     arcinit.obj
 0001:0001b3e8       ??_C@_0CJ@JHBMKCEI@leaving?5FindAdapter?5?9?5PCI?5Id?5not@FNODOBFM@ 0041c3e8     arcinit.obj
 0001:0001b412       ??_C@_0CL@HDBMPJMP@?$CK?5leaving?5FindAdapter?5?9?5PCI?5Id?5n@FNODOBFM@ 0041c412     arcinit.obj
 0001:0001b43e       ??_C@_0CH@LNPKNDMP@Rx?3?5BAR0?5Range?50x?$CFlx?5MappedSize?5@FNODOBFM@ 0041c43e     arcinit.obj
 0001:0001b466       ??_C@_0DF@OFCBAPFL@leaving?5FindAdapter?5?9?5fail?5mappi@FNODOBFM@ 0041c466     arcinit.obj
 0001:0001b49c       ??_C@_0DH@MNDLADLD@?$CK?5leaving?5FindAdapter?5?9?5fail?5map@FNODOBFM@ 0041c49c     arcinit.obj
 0001:0001b4d4       ??_C@_0DC@NODBFDAD@leaving?5FindAdapter?5?9?5illegal?5FW@FNODOBFM@ 0041c4d4     arcinit.obj
 0001:0001b506       ??_C@_0EH@FLDBENFC@?$CK?5leaving?5FindAdapter?5?9?5illegal?5@FNODOBFM@ 0041c506     arcinit.obj
 0001:0001b54e       ??_C@_0CK@GPLIPCCC@?$CK?5FULL?564?5BIT?5addressing?5support@FNODOBFM@ 0041c54e     arcinit.obj
 0001:0001b578       ??_C@_0CD@NJEIKDOH@?$CK?5New?5outstanding?5number?5chose?3?$CF@FNODOBFM@ 0041c578     arcinit.obj
 0001:0001b59c       ??_C@_0CD@CCLGIJ@?$CK?5Old?5outstanding?5number?5chose?3?$CF@FNODOBFM@ 0041c59c     arcinit.obj
 0001:0001b5c0       ??_C@_05JGHMLIKJ@devqd?$AA@FNODOBFM@ 0041c5c0     arcinit.obj
 0001:0001b5c6       ??_C@_0O@EPNNFPIH@?$CK?5DEV?5QD?3?5?$CFd?6?$AA@FNODOBFM@ 0041c5c6     arcinit.obj
 0001:0001b5d4       ??_C@_0N@OEGLNJCG@ioctlbufsize?$AA@FNODOBFM@ 0041c5d4     arcinit.obj
 0001:0001b5e2       ??_C@_0CI@LFOBEGIG@?$CK?5This?5is?564?9bit?5Vista?5or?5Longho@FNODOBFM@ 0041c5e2     arcinit.obj
 0001:0001b60a       ??_C@_0DB@NLEKMFMO@?$CK?5This?5is?532?9bit?5WS03?5R2?0?5Vista?5@FNODOBFM@ 0041c60a     arcinit.obj
 0001:0001b63c       ??_C@_0CA@DJAEOOFI@?$CK?5This?5is?564?9bit?5WS03?5SP1?5?4?4?4?5?6?$AA@FNODOBFM@ 0041c63c     arcinit.obj
 0001:0001b65c       ??_C@_0CA@IELABMFO@?$CK?5This?5is?532?9bit?5WS03?5SP1?5?4?4?4?5?6?$AA@FNODOBFM@ 0041c65c     arcinit.obj
 0001:0001b67c       ??_C@_0CA@MNGBKCLD@?$CK?5This?5is?532?9bit?5WS03?5RTM?5?4?4?4?5?6?$AA@FNODOBFM@ 0041c67c     arcinit.obj
 0001:0001b69c       ??_C@_0BL@FPDNGGII@?$CK?5Adapter?5is?5in?5poll?5mode?6?$AA@FNODOBFM@ 0041c69c     arcinit.obj
 0001:0001b6b8       ??_C@_0CO@NGAJFGIM@?$CK?5pDeviceExtension?9?$DONewCommInter@FNODOBFM@ 0041c6b8     arcinit.obj
 0001:0001b6e6       ??_C@_0CE@MCFGELJ@?$CK?5pDeviceExtension?9?$DOVendorId?3?50x@FNODOBFM@ 0041c6e6     arcinit.obj
 0001:0001b70a       ??_C@_0CE@PNKCKBKJ@?$CK?5pDeviceExtension?9?$DODeviceId?3?50x@FNODOBFM@ 0041c70a     arcinit.obj
 0001:0001b72e       ??_C@_0CH@NNKEKBEL@?$CK?5pDeviceExtension?9?$DOSubVendorId?3@FNODOBFM@ 0041c72e     arcinit.obj
 0001:0001b756       ??_C@_0CH@BEBMHIHH@?$CK?5pDeviceExtension?9?$DOSubSystemId?3@FNODOBFM@ 0041c756     arcinit.obj
 0001:0001b77e       ??_C@_0CB@ELGCJIGA@?$CK?5Uncached?5Memory?5address?3?50x?$CFp?6@FNODOBFM@ 0041c77e     arcinit.obj
 0001:0001b7a0       ??_C@_0CH@CKCEEBMD@?$CK?5Uncached?5Memory?5allocated?3?50x?$CF@FNODOBFM@ 0041c7a0     arcinit.obj
 0001:0001b7c8       ??_C@_0DK@INJPNBCP@?$CK?5MailBox?51?3?$CFx?0?5MailBox?52?3?$CFx?0?5Ma@FNODOBFM@ 0041c7c8     arcinit.obj
 0001:0001b802       ??_C@_0DB@DBAPOAM@?$CK?5pDeviceExtension?9?$DOMaxOutstandi@FNODOBFM@ 0041c802     arcinit.obj
 0001:0001b834       ??_C@_0DF@CKKIGFIG@?$CK?5pDeviceExtension?9?$DOMaxMSIXVecto@FNODOBFM@ 0041c834     arcinit.obj
 0001:0001b86a       ??_C@_0BA@EOIIECBM@loopbacklatency?$AA@FNODOBFM@ 0041c86a     arcinit.obj
 0001:0001b87a       ??_C@_0BC@BDCJEMN@?$CK?5FORCE?5INTX?3?5?$CFd?6?$AA@FNODOBFM@ 0041c87a     arcinit.obj
 0001:0001b88c       ??_C@_0BF@FJIEGFMA@?$CK?5FORCE?5POLLING?3?5?$CFd?6?$AA@FNODOBFM@ 0041c88c     arcinit.obj
 0001:0001b8a2       ??_C@_06DCBAGJIF@vecnum?$AA@FNODOBFM@ 0041c8a2     arcinit.obj
 0001:0001b8aa       ??_C@_0BK@NKHDFADJ@?$CK?5CPU?5Group?5number?5is?5?$CFd?6?$AA@FNODOBFM@ 0041c8aa     arcinit.obj
 0001:0001b8c4       ??_C@_0BJ@OBKJCBPL@?$CK?5CPU?5Node?5number?5is?5?$CFd?6?$AA@FNODOBFM@ 0041c8c4     arcinit.obj
 0001:0001b8de       ??_C@_0EB@PLAOEAEF@?$CK?5Valid_MSIX_Vectors?5is?5reset?5to@FNODOBFM@ 0041c8de     arcinit.obj
 0001:0001b920       ??_C@_0CN@KPEBIFEO@?$CK?5?$DN?$DN?$DN?$DN?$DN?$DN?$DO?5Final?5Vector?5Number?5is@FNODOBFM@ 0041c920     arcinit.obj
 0001:0001b94e       ??_C@_0CI@BJJEDHMG@?$CK?5pDeviceExtension?9?$DOVectorCapaci@FNODOBFM@ 0041c94e     arcinit.obj
 0001:0001b976       ??_C@_0DE@JJAKLEJD@?$CK?5pDeviceExtension?9?$DOMSIXIoThrott@FNODOBFM@ 0041c976     arcinit.obj
 0001:0001b9aa       ??_C@_0DF@LMKAIIEG@?$CK?5pDeviceExtension?9?$DOMSIXIoThrott@FNODOBFM@ 0041c9aa     arcinit.obj
 0001:0001b9e0       ??_C@_0BI@KNCDOCH@?$CK?5Node?5per?5Group?5is?5?$CFd?6?$AA@FNODOBFM@ 0041c9e0     arcinit.obj
 0001:0001b9f8       ??_C@_0BH@FMFCFLGH@?$CK?5Core?5per?5Node?5is?5?$CFd?6?$AA@FNODOBFM@ 0041c9f8     arcinit.obj
 0001:0001ba10       ??_C@_0CC@CEGCGDDK@?$CK?5?$DN?$DN?$DN?$DN?$DN?$DN?$DO?5End?5of?5summary?5?$DM?$DN?$DN?$DN?$DN?$DN?$DN@FNODOBFM@ 0041ca10     arcinit.obj
 0001:0001ba32       ??_C@_0EC@KMMHNEKL@?$CK?5ConfigInfo?9?$DOHwMSInterruptRouti@FNODOBFM@ 0041ca32     arcinit.obj
 0001:0001ba74       ??_C@_0BH@CDLDBOJF@?$CK?5SrbExtensionSize?3?$CFx?6?$AA@FNODOBFM@ 0041ca74     arcinit.obj
 0001:0001ba8c       ??_C@_0EK@GNODIBNL@?$CK?5MiniARC?5Interface?5?9?5?5CommandSi@FNODOBFM@ 0041ca8c     arcinit.obj
 0001:0001bad6       ??_C@_0EL@HJMLPDNI@?$CK?5New?5Comm?5Interface?5?9?5?5CommandS@FNODOBFM@ 0041cad6     arcinit.obj
 0001:0001bb22       ??_C@_0CM@NKHNJDEG@leaving?5FindAdapter?5?9?5fail?5initi@FNODOBFM@ 0041cb22     arcinit.obj
 0001:0001bb4e       ??_C@_0CO@GHEIBKDI@?$CK?5leaving?5FindAdapter?5?9?5fail?5ini@FNODOBFM@ 0041cb4e     arcinit.obj
 0001:0001bb7c       ??_C@_1EA@GNKDGDHK@?$AAA?$AAd?$AAa?$AAp?$AAt?$AAe?$AAr?$AA?5?$AAg?$AAo?$AAt?$AA?5?$AAi?$AAn?$AAv?$AAa?$AAl?$AAi?$AAd?$AA?5?$AAh?$AAo?$AAs?$AAt?$AA?5?$AAw?$AAi?$AAn?$AAd?$AAo?$AAw?$AA?$AA@FNODOBFM@ 0041cb7c     arcinit.obj
 0001:0001bbbc       ??_C@_1EI@NELDFHEH@?$AAA?$AAd?$AAa?$AAp?$AAt?$AAe?$AAr?$AA?5?$AAd?$AAo?$AAe?$AAs?$AA?5?$AAn?$AAo?$AAt?$AA?5?$AAs?$AAu?$AAp?$AAp?$AAo?$AAr?$AAt?$AA?5?$AA4?$AAG?$AAB?$AA?5?$AAw?$AAi?$AAn@FNODOBFM@ 0041cbbc     arcinit.obj
 0001:0001bc04       ??_C@_0DC@BFHJHJOO@?$CK?5fail?5SynFibCT_SET_MINIARC_HOST@FNODOBFM@ 0041cc04     arcinit.obj
 0001:0001bc36       ??_C@_0CE@IADADNNA@?$CK?5Use?5MU?5Register?5for?5IOP_Reset?4@FNODOBFM@ 0041cc36     arcinit.obj
 0001:0001bc5a       ??_C@_0CJ@LHHNJCHI@?$CK?5Use?5inbound?5doorbell?5for?5IOP_R@FNODOBFM@ 0041cc5a     arcinit.obj
 0001:0001bc84       ??_C@_0DI@LGINDMLA@?$CK?5ERROR?3?5FW?5does?5not?5provide?5whi@FNODOBFM@ 0041cc84     arcinit.obj
 0001:0001bcbc       ??_C@_0BP@DJKPJIGJ@?$CK?5Ignore_IOP_Reset?5is?5set?5?4?4?4?6?$AA@FNODOBFM@ 0041ccbc     arcinit.obj
 0001:0001bcdc       ??_C@_0CK@LEDHDPPJ@?$CK?5Disk?5Power?5Management?5is?5suppo@FNODOBFM@ 0041ccdc     arcinit.obj
 0001:0001bd06       ??_C@_0CJ@PJOACPGJ@?$CK?5This?5firmware?5supports?5fast?5JB@FNODOBFM@ 0041cd06     arcinit.obj
 0001:0001bd30       ??_C@_0DB@HEHLEMPI@?$CK?5Controller?5Firmware?5supports?5S@FNODOBFM@ 0041cd30     arcinit.obj
 0001:0001bd62       ??_C@_0CI@CJPAOACI@?$CK?5Controller?5Firmware?5supports?52@FNODOBFM@ 0041cd62     arcinit.obj
 0001:0001bd8a       ??_C@_0BM@LNCHEOOO@?$CK?5Virtual?5B?1T?1L?5?$CI?$CFd?1?$CFd?1?$CFd?$CJ?6?$AA@FNODOBFM@ 0041cd8a     arcinit.obj
 0001:0001bda6       ??_C@_0DA@OBMGONKI@?$CK?5Driver?5got?5SUPPORTED_NATIVE_HB@FNODOBFM@ 0041cda6     arcinit.obj
 0001:0001bdd6       ??_C@_0DI@GIKAIFLA@?$CK?5Driver?5did?5not?5get?5SUPPORTED_N@FNODOBFM@ 0041cdd6     arcinit.obj
 0001:0001be0e       ??_C@_0BH@LMHJIEKF@?$CK?5ExposeNonDASD?5is?5?$CFx?6?$AA@FNODOBFM@ 0041ce0e     arcinit.obj
 0001:0001be26       ??_C@_0BB@JIKBMNNG@QueueDepthPerLun?$AA@FNODOBFM@ 0041ce26     arcinit.obj
 0001:0001be38       ??_C@_0N@GDDJMKFE@PauseIOLimit?$AA@FNODOBFM@ 0041ce38     arcinit.obj
 0001:0001be46       ??_C@_0O@LIIBGGCF@ResumeIOLimit?$AA@FNODOBFM@ 0041ce46     arcinit.obj
 0001:0001be54       ??_C@_0O@OKMDGJBG@ConvertSGList?$AA@FNODOBFM@ 0041ce54     arcinit.obj
 0001:0001be62       ??_C@_0BE@IIJOOEPG@QueueStartThreshold?$AA@FNODOBFM@ 0041ce62     arcinit.obj
 0001:0001be76       ??_C@_0BD@CEDPKLI@QueueDumpThreshold?$AA@FNODOBFM@ 0041ce76     arcinit.obj
 0001:0001be8a       ??_C@_0BA@NLIGFJMK@MaxIoSizeQueued?$AA@FNODOBFM@ 0041ce8a     arcinit.obj
 0001:0001be9a       ??_C@_0N@MLHJOFDC@QueueAllowed?$AA@FNODOBFM@ 0041ce9a     arcinit.obj
 0001:0001bea8       ??_C@_0BC@IEBJFOIJ@FlushSizeInBlocks?$AA@FNODOBFM@ 0041cea8     arcinit.obj
 0001:0001beba       ??_C@_0EA@OJJGPBKL@leaving?5FindAdapter?5?9?5fail?5Handl@FNODOBFM@ 0041ceba     arcinit.obj
 0001:0001befa       ??_C@_0EC@HNCBOCML@?$CK?5leaving?5FindAdapter?5?9?5fail?5Han@FNODOBFM@ 0041cefa     arcinit.obj
 0001:0001bf3c       ??_C@_09NBOIBGGK@EnableWMI?$AA@FNODOBFM@ 0041cf3c     arcinit.obj
 0001:0001bf46       ??_C@_0DH@OIMAJCMK@?$CK?5?9?5Driver?5version?5?$CFs?0?5adapter?5n@FNODOBFM@ 0041cf46     arcinit.obj
 0001:0001bf7e       ??_C@_0DF@NGIHOECA@?$CK?5?9?5Size?5of?5HwDevExt?$DN0x?$CFx?4?5Size?5@FNODOBFM@ 0041cf7e     arcinit.obj
 0001:0001bfb4       ??_C@_0IC@BPBMMOAO@?$CK?5?9?5Size?$CISrbExt?$CJ?$DN0x?$CFx?4?5sizeof?$CIFI@FNODOBFM@ 0041cfb4     arcinit.obj
 0001:0001c036       ??_C@_0CA@ENCHFGMA@?$CK?5?9?5reported?5Size?$CISrbExt?$CJ?$DN0x?$CFx?6?$AA@FNODOBFM@ 0041d036     arcinit.obj
 0001:0001c056       ??_C@_0BG@JAEBOKND@?$CK?5?9?5Done?5FindAdapter?6?$AA@FNODOBFM@ 0041d056     arcinit.obj
 0001:0001c06c       ??_C@_0FF@LMEIGAGF@?$CK?5?9?5ConfigInfo?9?$DOMaximumTransferL@FNODOBFM@ 0041d06c     arcinit.obj
 0001:0001c0c2       ??_C@_0CG@GOHAMHPA@leaving?5FindAdapter?5?9?5adapter?5fo@FNODOBFM@ 0041d0c2     arcinit.obj
 0001:0001c0e8       ??_C@_0BN@DGMFEGDN@entering?5GetElapsedSeconds?5?6?$AA@FNODOBFM@ 0041d0e8     arcinit.obj
 0001:0001c106       ??_C@_0DD@GOLHMOHG@leaving?5GetElapsedSeconds?5?9?5seco@FNODOBFM@ 0041d106     arcinit.obj
 0001:0001c13a       ??_C@_0CJ@KCPJKGH@entering?5IsAdapterReadyForConfig@FNODOBFM@ 0041d13a     arcinit.obj
 0001:0001c164       ??_C@_0DB@PNDBFHEI@IsAdapterReadyForConfigCommand?3?5@FNODOBFM@ 0041d164     arcinit.obj
 0001:0001c196       ??_C@_0CH@PFKKGKLP@IsAdapterReadyForConfigCommand?3?5@FNODOBFM@ 0041d196     arcinit.obj
 0001:0001c1be       ??_C@_0DJ@FMKIDFML@?$CK?5leaving?5IsAdapterReadyForConfi@FNODOBFM@ 0041d1be     arcinit.obj
 0001:0001c1f8       ??_C@_0CI@LLJGECEO@leaving?5IsAdapterReadyForConfigC@FNODOBFM@ 0041d1f8     arcinit.obj
 0001:0001c220       ??_C@_0BD@LJONEFCN@entering?5IOPReset?6?$AA@FNODOBFM@ 0041d220     arcinit.obj
 0001:0001c234       ??_C@_0EN@CPGMGMBD@?$CK?$CK?5Fail?5to?5iopreset?5the?5adapter?5@FNODOBFM@ 0041d234     arcinit.obj
 0001:0001c282       ??_C@_0GF@NGDIBMBA@?$CK?5Driver?5has?5been?5waiting?55?5seco@FNODOBFM@ 0041d282     arcinit.obj
 0001:0001c2e8       ??_C@_1CG@OOCCJMGE@?$AAI?$AAO?$AAP?$AA?5?$AAR?$AAE?$AAS?$AAE?$AAT?$AA?5?$AAd?$AAi?$AAs?$AAa?$AAb?$AAl?$AAe?$AAd?$AA?$AA@FNODOBFM@ 0041d2e8     arcinit.obj
 0001:0001c30e       ??_C@_1CC@HLNFBNCO@?$AAI?$AAO?$AAP?$AA?5?$AAR?$AAE?$AAS?$AAE?$AAT?$AA?5?$AAf?$AAa?$AAi?$AAl?$AAe?$AAd?$AA?$AA@FNODOBFM@ 0041d30e     arcinit.obj
 0001:0001c330       ??_C@_0DE@GCJLBNBN@?$CK?$CK?5Fail?5to?5iopreset?5the?5adapter?0@FNODOBFM@ 0041d330     arcinit.obj
 0001:0001c364       ??_C@_0BI@DKKBLGKC@?$CK?$CK?5IOPReset?5succeeded?4?6?$AA@FNODOBFM@ 0041d364     arcinit.obj
 0001:0001c37c       ??_C@_0DI@IBEPOJOB@?$CK?5Discard?5HOSTRRQ?5leftover?3?5msg?5@FNODOBFM@ 0041d37c     arcinit.obj
 0001:0001c3b4       ??_C@_0DB@MLPIECHL@?$CK?5Discard?5HOSTRRQ?5leftover?3?5inde@FNODOBFM@ 0041d3b4     arcinit.obj
 0001:0001c3e6       ??_C@_0DG@MCABGJKN@Driver?5should?5not?5work?5under?5MSI@FNODOBFM@ 0041d3e6     arcinit.obj
 0001:0001c41c       ??_C@_0DE@DDNIODIO@?$CK?5Set?5pInitStruct?9?$DONoOfMsiVector@FNODOBFM@ 0041d41c     arcinit.obj
 0001:0001c450       ??_C@_0BC@JKJGEENA@leaving?5IOPReset?6?$AA@FNODOBFM@ 0041d450     arcinit.obj
 0001:0001c462       ??_C@_0EN@EHHFOLPM@?$CK?$CK?5returned?5?$CFd?5SRB?5to?5OS?5at?5Retu@FNODOBFM@ 0041d462     arcinit.obj
 0001:0001c4b0       ??_C@_0BK@OLLEIHIC@?$CK?5Switching?5to?5MSIx?5mode?6?$AA@FNODOBFM@ 0041d4b0     arcinit.obj
 0001:0001c4ca       ??_C@_0BA@EAOKKBLN@?$CK?5MSIx?5Enabled?6?$AA@FNODOBFM@ 0041d4ca     arcinit.obj
 0001:0001c4da       ??_C@_0EB@JEEKIEDM@?$CK?5Set?5pInitStruct?9?$DONoOfMsiVector@FNODOBFM@ 0041d4da     arcinit.obj
 0001:0001c51c       ??_C@_0EA@DFHNCIMC@?$CK?5Set?5pInitStruct?9?$DONoOfMsiVector@FNODOBFM@ 0041d51c     arcinit.obj
 0001:0001c55c       ??_C@_0FP@EFJPBKEO@?$CK?5Valid?5Vector?$CI?$CFd?$CJ?0?5msix?5capabil@FNODOBFM@ 0041d55c     arcinit.obj
 0001:0001c5bc       ??_C@_0BE@OKKJEBLK@?$CK?5MSIX?5NOT?5Enabled?6?$AA@FNODOBFM@ 0041d5bc     arcinit.obj
 0001:0001c5d0       ??_C@_0ED@LLOJEJPI@leaving?5HandleAdapterGetConfig?5a@FNODOBFM@ 0041d5d0     arcinit.obj
 0001:0001c614       ??_C@_0EF@MHNEOFPB@?$CK?5leaving?5HandleAdapterGetConfig@FNODOBFM@ 0041d614     arcinit.obj
 0001:0001c65a       ??_C@_0DP@PECHNPGJ@leaving?5HandleAdapterGetConfig?5a@FNODOBFM@ 0041d65a     arcinit.obj
 0001:0001c69a       ??_C@_0EB@CHAPDLOA@?$CK?5leaving?5HandleAdapterGetConfig@FNODOBFM@ 0041d69a     arcinit.obj
 0001:0001c6dc       ??_C@_0EC@JNDOKFCE@leaving?5HandleAdapterCommitConfi@FNODOBFM@ 0041d6dc     arcinit.obj
 0001:0001c71e       ??_C@_0EE@HMHNBLOK@?$CK?5leaving?5HandleAdapterCommitCon@FNODOBFM@ 0041d71e     arcinit.obj
 0001:0001c762       ??_C@_0CE@FDDAIENL@entering?5HandleAdapterConfigIssu@FNODOBFM@ 0041d762     arcinit.obj
 0001:0001c786       ??_C@_0EG@EOLGKFDM@leaving?5HandleAdapterConfigIssue@FNODOBFM@ 0041d786     arcinit.obj
 0001:0001c7cc       ??_C@_0EI@BLLNCBDL@?$CK?5leaving?5HandleAdapterConfigIss@FNODOBFM@ 0041d7cc     arcinit.obj
 0001:0001c814       ??_C@_0EC@KFDDDOGD@leaving?5HandleAdapterConfigIssue@FNODOBFM@ 0041d814     arcinit.obj
 0001:0001c856       ??_C@_0EE@EEHAIAKN@?$CK?5leaving?5HandleAdapterConfigIss@FNODOBFM@ 0041d856     arcinit.obj
 0001:0001c89a       ??_C@_0EC@EGKDAAOP@leaving?5HandleAdapterConfigIssue@FNODOBFM@ 0041d89a     arcinit.obj
 0001:0001c8dc       ??_C@_0EE@KHOALOCB@?$CK?5leaving?5HandleAdapterConfigIss@FNODOBFM@ 0041d8dc     arcinit.obj
 0001:0001c920       ??_C@_0CD@FIHDJCJC@leaving?5HandleAdapterConfigIssue@FNODOBFM@ 0041d920     arcinit.obj
 0001:0001c944       ??_C@_0BK@LNIBADPE@?$CK?5Setting?5StatusBatching?6?$AA@FNODOBFM@ 0041d944     arcinit.obj
 0001:0001c95e       ??_C@_0EF@JDALIICL@?$CK?5Firmware?5should?5support?5ACI2?5i@FNODOBFM@ 0041d95e     arcinit.obj
 0001:0001c9a4       ??_C@_0CB@DDHFLEBF@?$CK?5FW?5sets?5KERNEL_UP_AND_RUNNING?6@FNODOBFM@ 0041d9a4     arcinit.obj
 0001:0001c9c6       ??_C@_0CC@HECBNNJJ@?$CK?5FW?5is?5ready?5for?5config?5command@FNODOBFM@ 0041d9c6     arcinit.obj
 0001:0001c9e8       ??_C@_0BJ@GODFBPEB@?$CK?5Get?5config?5from?5FW?5ok?6?$AA@FNODOBFM@ 0041d9e8     arcinit.obj
 0001:0001ca02       ??_C@_0BK@PANMBLHC@?$CK?5Commit?5config?5to?5FW?5ok?6?$AA@FNODOBFM@ 0041da02     arcinit.obj
 0001:0001ca1c       ??_C@_0CA@BDIKNGAL@?$CK?5INIT?5Structure?5sent?5to?5FW?5ok?6?$AA@FNODOBFM@ 0041da1c     arcinit.obj
 0001:0001ca3c       ??_C@_0EE@GNMBAHCA@?$CK?5Get?5FW?5debug?5buffer?5failed?0?5bu@FNODOBFM@ 0041da3c     arcinit.obj
 0001:0001ca80       ??_C@_0BH@FLOGONBD@?$CK?5?9?5Driver?5version?5?$CFs?6?$AA@FNODOBFM@ 0041da80     arcinit.obj
 0001:0001ca98       ??_C@_0BO@IEENCLHE@entering?5HwInitializeAdapter?6?$AA@FNODOBFM@ 0041da98     arcinit.obj
 0001:0001cab6       ??_C@_1CA@OFEHMOBK@?$AAB?$AAa?$AAd?$AA?5?$AAP?$AAo?$AAr?$AAt?$AA?5?$AAD?$AAr?$AAi?$AAv?$AAe?$AAr?$AA?$AA@FNODOBFM@ 0041dab6     arcinit.obj
 0001:0001cad6       ??_C@_0FM@FIFECPG@?$CK?5pDeviceExtension?9?$DOValid_MSIX_V@FNODOBFM@ 0041dad6     arcinit.obj
 0001:0001cb32       ??_C@_0EH@ONHPKJKD@?$CK?5StorPortGetMSIInfo?5returned?5Fa@FNODOBFM@ 0041db32     arcinit.obj
 0001:0001cb7a       ??_C@_0EC@KLPNNIKH@?$CK?5StorPortGetMSIInfo?5returned?5st@FNODOBFM@ 0041db7a     arcinit.obj
 0001:0001cbbc       ??_C@_0EE@OLLCNNAO@?$CK?5StorPortGetMSIInfo?5returned?5st@FNODOBFM@ 0041dbbc     arcinit.obj
 0001:0001cc00       ??_C@_0EJ@OBPFJGIJ@?$CK?5StorPortGetMSIInfo?5returned?5st@FNODOBFM@ 0041dc00     arcinit.obj
 0001:0001cc4a       ??_C@_0CF@FDBIIPFF@?$CK?5This?5Tupelo?5driver?5is?5MSI?5enab@FNODOBFM@ 0041dc4a     arcinit.obj
 0001:0001cc70       ??_C@_0BO@FHHBMMGN@?$CK?5PerfConfigData?4Flags?3?50x?$CFx?6?$AA@FNODOBFM@ 0041dc70     arcinit.obj
 0001:0001cc8e       ??_C@_0FE@LBLIGLIO@GetDoorbellMaskForIOPReset?5retur@FNODOBFM@ 0041dc8e     arcinit.obj
 0001:0001cce2       ??_C@_0DN@IMFNPMPP@?$CK?5Failed?5to?5Initialize?5Adapter?5i@FNODOBFM@ 0041dce2     arcinit.obj
 0001:0001cd20       ??_C@_0DE@CMNGFMDL@?$CK?5Succeed?5to?5Initialize?5Adapter?5@FNODOBFM@ 0041dd20     arcinit.obj
 0001:0001cd54       ??_C@_0EG@KGJBNOFG@?$CK?5Failed?5to?5Initialize?5Adapter?5i@FNODOBFM@ 0041dd54     arcinit.obj
 0001:0001cd9a       ??_C@_0BP@MCCOMIEF@?$CK?5leaving?5HwInitializeAdapter?6?$AA@FNODOBFM@ 0041dd9a     arcinit.obj
 0001:0001cdba       ??_C@_0FN@OJHBJJGK@?$CK?5StorPortAllocateContiguousMemo@FNODOBFM@ 0041ddba     arcinit.obj
 0001:0001ce18       ??_C@_0FD@MKBBGMOP@?$CK?5PROBLEM?3?5returnedSize?5?$DN?50?5?$CISto@FNODOBFM@ 0041de18     arcinit.obj
 0001:0001ce6c       ??_C@_0IH@LCJNFDMG@?$CK?5StorPortAllocateContiguousMemo@FNODOBFM@ 0041de6c     arcinit.obj
 0001:0001cef4       ??_C@_0BI@BOGNCAIA@entering?5InitializeDPC?6?$AA@FNODOBFM@ 0041def4     arcinit.obj
 0001:0001cf0c       ??_C@_0BL@ICGKMMAJ@?$CK?5Start?5scanning?5group?5?$CFd?6?$AA@FNODOBFM@ 0041df0c     arcinit.obj
 0001:0001cf28       ??_C@_0CO@FDNLALKJ@?$CK?5Group?5Affinity?5for?5msix?5vector@FNODOBFM@ 0041df28     arcinit.obj
 0001:0001cf56       ??_C@_0DA@FPNPLEPN@?$CK?5NUMA?5node?5for?5MSIX?5vector?5?$CFd?5i@FNODOBFM@ 0041df56     arcinit.obj
 0001:0001cf86       ??_C@_0DP@MAPFHEEH@?$CK?5Outbound?5Queue?5Memory?5allocate@FNODOBFM@ 0041df86     arcinit.obj
 0001:0001cfc6       ??_C@_0CG@GFDFODNM@?$CK?5MemoryBlock?5?$CFd?5assigned?5in?5nod@FNODOBFM@ 0041dfc6     arcinit.obj
 0001:0001cfec       ??_C@_0DG@CGCBEMEO@?$CK?5MSG?5CAP?5setup?5failed?5?$CIbecause?5@FNODOBFM@ 0041dfec     arcinit.obj
 0001:0001d022       ??_C@_0ED@CJAGENOE@?$CK?5we?5are?5processing?5last?5MSIX?5ve@FNODOBFM@ 0041e022     arcinit.obj
 0001:0001d066       ??_C@_0HA@GKDMKHHO@?$CK?5we?5have?5a?5problem?4?5All?5groups?1@FNODOBFM@ 0041e066     arcinit.obj
 0001:0001d0d6       ??_C@_0FD@LFCJJKMC@?$CK?5StorPortGetLogicalProcessorRel@FNODOBFM@ 0041e0d6     arcinit.obj
 0001:0001d12a       ??_C@_0BG@FAIHHGLA@?$CK?5Vector?5?$CFd?5is?5done?6?6?$AA@FNODOBFM@ 0041e12a     arcinit.obj
 0001:0001d140       ??_C@_0DJ@MGMHFMAN@?$CK?5Failed?5to?5Initialize?5Adapter?5i@FNODOBFM@ 0041e140     arcinit.obj
 0001:0001d17a       ??_C@_0DA@GDJCAINB@?$CK?5Succeed?5to?5Initialize?5Adapter?5@FNODOBFM@ 0041e17a     arcinit.obj
 0001:0001d1aa       ??_C@_0BJ@CFFELFMJ@?$CK?5MSIx?5DPCs?5initialized?6?$AA@FNODOBFM@ 0041e1aa     arcinit.obj
 0001:0001d1c4       ??_C@_0BI@LAPEOFCN@?$CK?5?9?5Done?5InitializeDPC?6?$AA@FNODOBFM@ 0041e1c4     arcinit.obj
 0001:0001d1dc       ??_C@_0BH@PAHICDNJ@leaving?5InitializeDPC?6?$AA@FNODOBFM@ 0041e1dc     arcinit.obj
 0001:0001d1f4       ??_C@_0CP@OJKLKHLO@entering?5InitializeConsumerProdu@FNODOBFM@ 0041e1f4     arcinit.obj
 0001:0001d224       ??_C@_0DE@MJJEGAKI@leaving?5InitializeConsumerProduc@FNODOBFM@ 0041e224     arcinit.obj
 0001:0001d258       ??_C@_0CO@NEGLFCOP@leaving?5InitializeConsumerProduc@FNODOBFM@ 0041e258     arcinit.obj
 0001:0001d286       ??_C@_0CP@IKCNDLML@entering?5InitializeConsumerProdu@FNODOBFM@ 0041e286     arcinit.obj
 0001:0001d2b6       ??_C@_0DF@IICIHNDP@leaving?5InitializeConsumerProduc@FNODOBFM@ 0041e2b6     arcinit.obj
 0001:0001d2ec       ??_C@_0DE@OBANPGHF@leaving?5InitializeConsumerProduc@FNODOBFM@ 0041e2ec     arcinit.obj
 0001:0001d320       ??_C@_0CP@GDFIJJML@entering?5InitializeMessageUnitQu@FNODOBFM@ 0041e320     arcinit.obj
 0001:0001d350       ??_C@_0DF@CLHHLLI@leaving?5InitializeMessageUnitQue@FNODOBFM@ 0041e350     arcinit.obj
 0001:0001d386       ??_C@_0DE@BBDIIBAC@leaving?5InitializeMessageUnitQue@FNODOBFM@ 0041e386     arcinit.obj
 0001:0001d3ba       ??_C@_0BI@PNFIHJKN@entering?5MapDeviceBase?6?$AA@FNODOBFM@ 0041e3ba     arcinit.obj
 0001:0001d3d2       ??_C@_1CM@FGGDGCGC@?$AAA?$AAd?$AAa?$AAp?$AAt?$AAe?$AAr?$AA?5?$AAb?$AAo?$AAo?$AAt?$AA?5?$AAt?$AAi?$AAm?$AAe?$AA?5?$AAo?$AAu?$AAt?$AA?$AA@FNODOBFM@ 0041e3d2     arcinit.obj
 0001:0001d3fe       ??_C@_0CO@NHBGNFPE@?$CK?5Driver?5got?564?5bit?5FIB?5support?5@FNODOBFM@ 0041e3fe     arcinit.obj
 0001:0001d42c       ??_C@_0DG@EECBHNEJ@?$CK?5Driver?5did?5not?5get?564?5bit?5FIB?5@FNODOBFM@ 0041e42c     arcinit.obj
 0001:0001d462       ??_C@_0CB@MHHOKKDH@?$CK?5Smart?5Array?5Based?5FW?5detected?6@FNODOBFM@ 0041e462     arcinit.obj
 0001:0001d484       ??_C@_0CG@INGLDPEA@?$CK?5This?5is?5NOT?5a?5Smart?5Array?5Base@FNODOBFM@ 0041e484     arcinit.obj
 0001:0001d4aa       ??_C@_0DL@HHJHAPNC@?$CK?5StorPortGetDeviceBase?5failed?0?5@FNODOBFM@ 0041e4aa     arcinit.obj
 0001:0001d4e6       ??_C@_0FM@FAGAFMJI@?$CK?5StorPortGetDeviceBaseB1?5failed@FNODOBFM@ 0041e4e6     arcinit.obj
 0001:0001d542       ??_C@_0FM@DFFNMELK@?$CK?5StorPortGetDeviceBaseB0?5failed@FNODOBFM@ 0041e542     arcinit.obj
 0001:0001d59e       ??_C@_0DH@GMHBCEJM@?$CK?5GET_MINIARC_PROPERTIES?5fails?0?5@FNODOBFM@ 0041e59e     arcinit.obj
 0001:0001d5d6       ??_C@_0CE@JIIGOPEA@?$CK?5This?5is?5a?5BEDROC?5inplementatio@FNODOBFM@ 0041e5d6     arcinit.obj
 0001:0001d5fa       ??_C@_0CF@HKNELPOC@leaving?5MapDeviceBase?5?9?5rtnval?5?$DN@FNODOBFM@ 0041e5fa     arcinit.obj
 0001:0001d620       ??_C@_0BG@LOIMFNHP@entering?5MatchPciIds?6?$AA@FNODOBFM@ 0041e620     arcinit.obj
 0001:0001d636       ??_C@_08HNOCAICB@Adaptec?5?$AA@FNODOBFM@ 0041e636     arcinit.obj
 0001:0001d640       ??_C@_0FA@LPOMHBHK@?$CK?5leaving?5MatchPciIds?0?5rtnval?5?$DN?5@FNODOBFM@ 0041e640     arcinit.obj
 0001:0001d690       ??_C@_0FA@BIGBANAO@?$CK?5leaving?5MatchPciIds?0?5rtnval?5?$DN?5@FNODOBFM@ 0041e690     arcinit.obj
 0001:0001d6e0       ??_C@_0CC@GEDCIDMJ@leaving?5MatchPciIds?0?5rtnval?5?$DN?5?$CFx@FNODOBFM@ 0041e6e0     arcinit.obj
 0001:0001d702       ??_C@_0DG@MJCHKBMN@?$CK?5Calling?5CompleteBufferedReques@FNODOBFM@ 0041e702     arcinit.obj
 0001:0001d738       ??_C@_0HF@LDMKNKBL@?$CK?5Calling?5DequeueRawIoReadWriteR@FNODOBFM@ 0041e738     arcinit.obj
 0001:0001d7ae       ??_C@_0DO@HDLNLCMA@?$CK?5Calling?5CompleteAllSortingQueu@FNODOBFM@ 0041e7ae     arcinit.obj
 0001:0001d7ec       ??_C@_0CG@EHFONFB@ReturningLocalOutstandingRequest@FNODOBFM@ 0041e7ec     arcinit.obj
 0001:0001d812       ??_C@_0CL@CGNJGHDF@?$CK?5?$CFd?5outstanding?5IO?5left?5after?5c@FNODOBFM@ 0041e812     arcinit.obj
 0001:0001d83e       ??_C@_0CF@IKJOOFLA@?$CK?5ResetAdapter?3?5Entering?5Routine@FNODOBFM@ 0041e83e     arcinit.obj
 0001:0001d864       ??_C@_0FI@OABPGHMC@?$CK?5ResetAdapter?3?5FW?5is?5processing@FNODOBFM@ 0041e864     arcinit.obj
 0001:0001d8bc       ??_C@_0DK@DMNFFNOF@?$CK?5ResetAdapter?3?5OS?5calls?5ResetAd@FNODOBFM@ 0041e8bc     arcinit.obj
 0001:0001d8f6       ??_C@_0CE@IFPMEIEL@?$CK?5ResetAdapter?3?5BlinLed?5Code?3?50x@FNODOBFM@ 0041e8f6     arcinit.obj
 0001:0001d91a       ??_C@_1CE@ENBAPEOO@?$AAB?$AAl?$AAi?$AAn?$AAk?$AAL?$AAE?$AAD?$AA?5?$AAd?$AAe?$AAt?$AAe?$AAc?$AAt?$AAe?$AAd?$AA?$AA@FNODOBFM@ 0041e91a     arcinit.obj
 0001:0001d93e       ??_C@_0CL@MJAGNJPB@?$CK?5ResetAdapter?3?5IOP?5RESET?5due?5to@FNODOBFM@ 0041e93e     arcinit.obj
 0001:0001d96a       ??_C@_0DG@CLNGJPOA@?$CK?5ResetAdapter?3?5SendSynchFib?5fai@FNODOBFM@ 0041e96a     arcinit.obj
 0001:0001d9a0       ??_C@_0FF@JLPFKNGK@?$CK?5ResetAdapter?3?5There?5is?5a?5pendi@FNODOBFM@ 0041e9a0     arcinit.obj
 0001:0001d9f6       ??_C@_0EC@MMLNJELN@?$CK?5ResetAdapter?3?5set?5TriggerIOPRe@FNODOBFM@ 0041e9f6     arcinit.obj
 0001:0001da38       ??_C@_0EH@BGKKNIMJ@?$CK?5ResetAdapter?3?5synch?5command?5Re@FNODOBFM@ 0041ea38     arcinit.obj
 0001:0001da80       ??_C@_0EE@KPCKIKGP@?$CK?5ResetAdapter?3?5AdapterIsAlive?5r@FNODOBFM@ 0041ea80     arcinit.obj
 0001:0001dac4       ??_C@_0DN@OJOIDCGM@?$CK?5ResetAdapter?3?5leaving?5Routine?5@FNODOBFM@ 0041eac4     arcinit.obj
 0001:0001db02       ??_C@_0DN@MKLLHNDH@?$CK?5ResetAdapter?3?5IOP?5RESET?5due?5to@FNODOBFM@ 0041eb02     arcinit.obj
 0001:0001db40       ??_C@_0DA@IHJFMKGH@?$CK?5ResetAdapter?3?5IOP?5RESET?5due?5to@FNODOBFM@ 0041eb40     arcinit.obj
 0001:0001db70       ??_C@_0FK@LPHHHNGK@?$CK?5ResetAdapter?3?5device?5on?5path?54@FNODOBFM@ 0041eb70     arcinit.obj
 0001:0001dbca       ??_C@_0EG@FKMCGCCN@?$CK?5ResetAdapter?3?5IOP?5RESET?5due?5to@FNODOBFM@ 0041ebca     arcinit.obj
 0001:0001dc10       ??_C@_0DE@IDNFNJBF@?$CK?5ResetAdapter?3?5NO?5lun?5reset?5cou@FNODOBFM@ 0041ec10     arcinit.obj
 0001:0001dc44       ??_C@_0DM@KJNOMFJC@?$CK?5ResetAdapter?3?5leaving?5Routine?0@FNODOBFM@ 0041ec44     arcinit.obj
 0001:0001dc80       ??_C@_0EK@OOPLAGOO@?$CK?5ResetAdapter?3?5set?5timer?5to?5che@FNODOBFM@ 0041ec80     arcinit.obj
 0001:0001dcca       ??_C@_0DM@LMPLKKMJ@?$CK?5ResetAdapter?3?5leaving?5Routine?5@FNODOBFM@ 0041ecca     arcinit.obj
 0001:0001dd06       ??_C@_0EJ@DNGMPOBO@?$CK?5ResetAdapter?3?5HWSoftReset?5leav@FNODOBFM@ 0041ed06     arcinit.obj
 0001:0001dd50       ??_C@_0BH@KIKHJKLE@?$DMHW?$DOTD?$AI?$AA?$AA?$AA?$AA?$AA?$AA?$AA?$AA?$AADW?$AA?$AAZZ?$AA@FNODOBFM@ 0041ed50     arcinit.obj
 0001:0001dd68       ??_C@_0BP@BFNIMKLC@?$CK?5SetFwTime?3?5Time?5sent?5failed?6?$AA@FNODOBFM@ 0041ed68     arcinit.obj
 0001:0001dd88       ??_C@_0BL@IIHDOJJO@?$CK?5Time?3?5?$CFd?4?$CFd?4?$CFd?5?$CFd?3?$CFd?3?$CFd?6?$AA@FNODOBFM@ 0041ed88     arcinit.obj
 0001:0001dda4       ??_C@_0BG@NCOEMLFM@?$CK?5Driver?5version?5?$CFs?5?6?$AA@FNODOBFM@ 0041eda4     arcinit.obj
 0001:0001ddba       ??_C@_0CF@KGAABJAP@?$CK?5SetFwTime?3?5Time?5sent?5successfu@FNODOBFM@ 0041edba     arcinit.obj
 0001:0001dde0       ??_C@_0DN@BMDNNOBN@?$CK?5GetThorHbaPhyDevInfo?3?5synch?5FI@FNODOBFM@ 0041ede0     arcinit.obj
 0001:0001de1e       ??_C@_0FG@PNEDCHMO@?$CK?5one?5dual?5port?5entry?5?$CIB?1T?1nexus@FNODOBFM@ 0041ee1e     arcinit.obj
 0001:0001de74       ??_C@_0EM@BKPAJHPD@?$CK?5One?5entry?5?$CIB?1T?1nexus?3?5?$CFd?1?$CFd?10x@FNODOBFM@ 0041ee74     arcinit.obj
 0001:0001dec0       ??_C@_0BI@NKGGGHHE@?$CK?5?$CFd?5HBA?5devices?5found?6?$AA@FNODOBFM@ 0041eec0     arcinit.obj
 0001:0001ded8       ??_C@_0DD@PLCLGMJE@?$CK?5All?5HBA?5devices?8?5average?5Queue@FNODOBFM@ 0041eed8     arcinit.obj
 0001:0001df0c       ??_C@_0BF@GFOGGOIF@GetThorHbaPhyDevInfo?$AA@FNODOBFM@ 0041ef0c     arcinit.obj
 0001:0001df22       ??_C@_0CL@OHPEFDNF@?$CK?5There?5is?5a?5synch?5SRB?5pending?0?5@FNODOBFM@ 0041ef22     arcinit.obj
 0001:0001df4e       ??_C@_0DJ@HDKNIPML@?$CK?5Not?5a?5Thor?5product?5OR?5virtual?5@FNODOBFM@ 0041ef4e     arcinit.obj
 0001:0001df88       ??_C@_1FE@PCKFJNFD@?$AAR?$AAe?$AAs?$AAe?$AAt?$AA?5?$AAf?$AAr?$AAo?$AAm?$AA?5?$AAO?$AAS?$AA?3?$AAp?$AAa?$AAt?$AAh?$AA?5?$AA?$CD?$AA?5?$AA?5?$AA?0?$AAo?$AAu?$AAt?$AAs?$AAt?$AAa?$AAn?$AAd?$AAi@FNODOBFM@ 0041ef88     arcinit.obj
 0001:0001dfdc       ??_C@_1FC@CLHIPIHG@?$AAG?$AAo?$AAt?$AA?5?$AAL?$AAU?$AAN?$AA?5?$AAR?$AAE?$AAS?$AAE?$AAT?$AA?5?$AAf?$AAo?$AAr?$AA?5?$AAp?$AAa?$AAt?$AAh?$AA?5?$AA?$CD?$AA?5?$AA?5?$AA?0?$AA?5?$AAt?$AAa?$AAr?$AAg@FNODOBFM@ 0041efdc     arcinit.obj
 0001:0001e02e       ??_C@_1FI@HJHKOPPE@?$AAG?$AAo?$AAt?$AA?5?$AAT?$AAa?$AAr?$AAg?$AAe?$AAt?$AA?5?$AAR?$AAE?$AAS?$AAE?$AAT?$AA?5?$AAf?$AAo?$AAr?$AA?5?$AAp?$AAa?$AAt?$AAh?$AA?5?$AA?$CD?$AA?5?$AA?5?$AA?0?$AA?5?$AAt@FNODOBFM@ 0041f02e     arcinit.obj
 0001:0001e086       ??_C@_1EC@DEFLMBHE@?$AAI?$AAO?$AAP?$AA?5?$AAR?$AAE?$AAS?$AAE?$AAT?$AA?5?$AAb?$AAe?$AAc?$AAa?$AAu?$AAs?$AAe?$AA?5?$AAo?$AAf?$AA?5?$AAF?$AAW?$AA?5?$AAB?$AAl?$AAi?$AAn?$AAk?$AAL?$AAE?$AAD@FNODOBFM@ 0041f086     arcinit.obj
 0001:0001e0c8       ??_C@_1FA@GLBMBCFD@?$AAR?$AAe?$AAq?$AAu?$AAe?$AAs?$AAt?$AAA?$AAd?$AAa?$AAp?$AAt?$AAe?$AAr?$AAI?$AAn?$AAf?$AAo?$AA?5?$AAp?$AAe?$AAn?$AAd?$AAi?$AAn?$AAg?$AA?5?$AA?5?$AA?5?$AA?5?$AA?5?$AA?5@FNODOBFM@ 0041f0c8     arcinit.obj
 0001:0001e118       ??_C@_1EK@DPFNMDNI@?$AAI?$AAO?$AAP?$AAR?$AAE?$AAS?$AAE?$AAT?$AA?3?$AA?5?$AAR?$AAe?$AAq?$AAu?$AAe?$AAs?$AAt?$AAA?$AAd?$AAa?$AAp?$AAt?$AAe?$AAr?$AAI?$AAn?$AAf?$AAo?$AA?5?$AAt?$AAi?$AAm@FNODOBFM@ 0041f118     arcinit.obj
 0001:0001e162       ??_C@_1EC@JONMGECF@?$AAR?$AAA?$AA?3?$AA?5?$AAA?$AAd?$AAa?$AAp?$AAt?$AAe?$AAr?$AAI?$AAs?$AAA?$AAl?$AAi?$AAv?$AAe?$AA?5?$AAr?$AAe?$AAt?$AAu?$AAr?$AAn?$AAs?$AA?5?$AAf?$AAa?$AAl?$AAs?$AAe@FNODOBFM@ 0041f162     arcinit.obj
 0001:0001e1a4       ??_C@_1EA@KMCOFCE@?$AAI?$AAO?$AAP?$AA?5?$AAR?$AAE?$AAS?$AAE?$AAT?$AA?5?$AAf?$AAo?$AAr?$AA?5?$AAS?$AAm?$AAa?$AAr?$AAt?$AAH?$AAB?$AAA?$AA?5?$AAp?$AAa?$AAt?$AAh?$AA?5?$AA?$CD?$AA?5?$AA?5?$AA?$AA@FNODOBFM@ 0041f1a4     arcinit.obj
 0001:0001e1e4       ??_C@_1EK@EBJJOFBF@?$AAR?$AAE?$AAS?$AAE?$AAT?$AA?$CI?$AAc?$AAn?$AAt?$AA?$DO?$AA?$DN?$AA5?$AA?$CJ?$AA?3?$AA?5?$AAp?$AAa?$AAt?$AAh?$AA?5?$AA?$CD?$AA?5?$AA?5?$AA?0?$AA?5?$AAt?$AAa?$AAr?$AAg?$AAe?$AAt?$AA?5@FNODOBFM@ 0041f1e4     arcinit.obj
 0001:0001e22e       ??_C@_1DA@EFMGPIMG@?$AAS?$AAO?$AAF?$AAT?$AA?5?$AAR?$AAE?$AAS?$AAE?$AAT?$AA?5?$AAI?$AAs?$AAs?$AAu?$AAe?$AAd?$AA?5?$AAt?$AAo?$AA?5?$AAF?$AAW?$AA?$AA@FNODOBFM@ 0041f22e     arcinit.obj
 0001:0001e25e       ??_C@_1CO@GBDEAPLE@?$AAI?$AAO?$AAP?$AA?5?$AAR?$AAE?$AAS?$AAE?$AAT?$AA?5?$AAI?$AAs?$AAs?$AAu?$AAe?$AAd?$AA?5?$AAt?$AAo?$AA?5?$AAF?$AAW?$AA?$AA@FNODOBFM@ 0041f25e     arcinit.obj
 0001:0001e28c       ??_C@_1EI@KMCCOKBI@?$AAF?$AAW?$AA?5?$AAK?$AAE?$AAR?$AAN?$AAE?$AAL?$AA?5?$AAP?$AAA?$AAN?$AAI?$AAC?$AA?5?$AAD?$AAe?$AAt?$AAe?$AAc?$AAt?$AAe?$AAd?$AA?0?$AA?5?$AAB?$AAL?$AAE?$AAD?$AA?5?$AA?$CD@FNODOBFM@ 0041f28c     arcinit.obj
 0001:0001e2d4       ??_C@_1GC@LLIAMOBH@?$AAD?$AAr?$AAi?$AAv?$AAe?$AAr?$AA?5?$AAI?$AAn?$AAi?$AAt?$AA?3?$AAF?$AAW?$AA?5?$AAN?$AAo?$AAt?$AA?5?$AAU?$AAp?$AA?5?$AA?$CG?$AA?5?$AAR?$AAu?$AAn?$AAn?$AAi?$AAn?$AAg?$AA?0@FNODOBFM@ 0041f2d4     arcinit.obj
 0001:0001e336       ??_C@_1GA@EMDMIJOE@?$AAD?$AAr?$AAi?$AAv?$AAe?$AAr?$AA?5?$AAI?$AAn?$AAi?$AAt?$AA?3?$AA?5?$AAC?$AAT?$AA_?$AAC?$AAO?$AAN?$AAF?$AAI?$AAG?$AA_?$AAS?$AAT?$AAA?$AAT?$AAU?$AAS?$AA_?$AAR?$AAE@FNODOBFM@ 0041f336     arcinit.obj
 0001:0001e396       ??_C@_1FM@HDDFDKHH@?$AAD?$AAr?$AAi?$AAv?$AAe?$AAr?$AA?5?$AAI?$AAn?$AAi?$AAt?$AA?3?$AA?5?$AAC?$AAT?$AA_?$AAG?$AAE?$AAT?$AA_?$AAC?$AAO?$AAN?$AAF?$AAI?$AAG?$AA_?$AAS?$AAT?$AAA?$AAT?$AAU@FNODOBFM@ 0041f396     arcinit.obj
 0001:0001e3f2       ??_C@_1FC@DDFGNEIP@?$AAD?$AAr?$AAi?$AAv?$AAe?$AAr?$AA?5?$AAI?$AAn?$AAi?$AAt?$AA?3?$AA?5?$AAC?$AAT?$AA_?$AAC?$AAO?$AAM?$AAM?$AAI?$AAT?$AA_?$AAC?$AAO?$AAN?$AAF?$AAI?$AAG?$AA?$CI?$AA?5?$AA?5@FNODOBFM@ 0041f3f2     arcinit.obj
 0001:0001e444       ??_C@_1GK@NIBLIOAN@?$AAD?$AAr?$AAi?$AAv?$AAe?$AAr?$AA?5?$AAI?$AAn?$AAi?$AAt?$AA?3?$AA?5?$AAA?$AAD?$AAA?$AAP?$AAT?$AAE?$AAR?$AA_?$AAI?$AAN?$AAI?$AAT?$AA_?$AAS?$AAT?$AAR?$AAU?$AAC?$AAT@FNODOBFM@ 0041f444     arcinit.obj
 0001:0001e4ae       ??_C@_1FG@JJEGPKHN@?$AAD?$AAr?$AAi?$AAv?$AAe?$AAr?$AA?5?$AAI?$AAn?$AAi?$AAt?$AA?3?$AA?5?$AAV?$AAM?$AA_?$AAC?$AAo?$AAn?$AAt?$AAa?$AAi?$AAn?$AAe?$AAr?$AAC?$AAo?$AAn?$AAf?$AAi?$AAg?$AA?$CI@FNODOBFM@ 0041f4ae     arcinit.obj
 0001:0001e504       ??_C@_1EM@EFNIIMIL@?$AAD?$AAr?$AAi?$AAv?$AAe?$AAr?$AA?5?$AAI?$AAn?$AAi?$AAt?$AA?3?$AA?5?$AAT?$AAi?$AAm?$AAe?$AAd?$AAo?$AAu?$AAt?$AA?0?$AA?5?$AAI?$AAn?$AAi?$AAt?$AA?5?$AAS?$AAt?$AAa?$AAg@FNODOBFM@ 0041f504     arcinit.obj
 0001:0001e550       ??_C@_0BG@HHGGAPDG@entering?5HWSoftReset?6?$AA@FNODOBFM@ 0041f550     arcinit.obj
 0001:0001e566       ??_C@_0CB@CNHAMPIN@HwSoftReset?3?5Soft?5Reset?5Issued?4?6@FNODOBFM@ 0041f566     arcinit.obj
 0001:0001e588       ??_C@_0DJ@CBPNBDFH@?$CK?5Set?5pInitStruct?9?$DONoOfMsiVector@FNODOBFM@ 0041f588     arcinit.obj
 0001:0001e5c2       ??_C@_0BG@FGBHCKJG@CompleteQueuedRequest?$AA@FNODOBFM@ 0041f5c2     cmddelivery.obj
 0001:0001e5d8       ??_C@_0DM@OFFCECMD@IN?5?$CFs?0?5WE?5ARE?5SEEING?5AIF?5FIB?4?5DO@FNODOBFM@ 0041f5d8     cmddelivery.obj
 0001:0001e614       ??_C@_0L@ENAJINDB@Management?$AA@FNODOBFM@ 0041f614     cmddelivery.obj
 0001:0001e620       ??_C@_0BB@JIADCMFJ@Array?5?5?5?5?5?5?5?5?5?5?5?$AA@FNODOBFM@ 0041f620     cmddelivery.obj
 0001:0001e632       ??_C@_08BFDLJAAH@ADAPTEC?5?$AA@FNODOBFM@ 0041f632     cmddelivery.obj
 0001:0001e63c       ??_C@_0BB@HJODFKJH@ARRAY?5?5?5?5?5?5?5?5?5?5?5?$AA@FNODOBFM@ 0041f63c     cmddelivery.obj
 0001:0001e64e       ??_C@_0CB@IIENMBOI@?$CK?5Got?5an?5AIF?5in?5crash?5dump?5mode?6@FNODOBFM@ 0041f64e     cmddelivery.obj
 0001:0001e670       ??_C@_0DO@NPBDNHBG@?$CK?5Should?5not?5be?5here?0?5we?5should?5@FNODOBFM@ 0041f670     cmddelivery.obj
 0001:0001e6ae       ??_C@_0CO@PDPAIINM@?$CK?5PollSmartHBAFIBCompletion?3?5wai@FNODOBFM@ 0041f6ae     cmddelivery.obj
 0001:0001e6dc       ??_C@_0FM@ENJACBOF@?$CK?5SCSIOP_SYNCHRONIZE_CACHE?$CICDM?$CJ?3@FNODOBFM@ 0041f6dc     cmddelivery.obj
 0001:0001e738       ??_C@_0GA@MEOEEOJH@?$CK?5SCSIOP_SYNCHRONIZE_CACHE?$CICDM?$CJ?3@FNODOBFM@ 0041f738     cmddelivery.obj
 0001:0001e798       ??_C@_0HI@CALKOMHC@?$CK?5SendSynchFib?3?5There?5is?5a?5pendi@FNODOBFM@ 0041f798     cmddelivery.obj
 0001:0001e810       ??_C@_0FM@IHOMFPBM@?$CK?5In?5StartIo?0?5FW?5is?5still?5NOT?5ba@FNODOBFM@ 0041f810     cmddelivery.obj
 0001:0001e86c       ??_C@_0CN@EPOHBMBH@?$CK?5path?5?$CFd?5target?5?$CFd?5reset?5counte@FNODOBFM@ 0041f86c     cmddelivery.obj
 0001:0001e89a       ??_C@_0CB@KIAHGGON@?5RESET?5is?5for?5Smart?5HBA?5device?5?6@FNODOBFM@ 0041f89a     cmddelivery.obj
 0001:0001e8bc       ??_C@_0BP@PAHACOBL@?$CK?5Got?5path?5?$CFd?5target?5?$CFd?5reset?6?$AA@FNODOBFM@ 0041f8bc     cmddelivery.obj
 0001:0001e8dc       ??_C@_0CC@BGHDODBG@?$CK?5SRB_FUNCTION_POWER?3?5action?3?5?$CFd@FNODOBFM@ 0041f8dc     cmddelivery.obj
 0001:0001e8fe       ??_C@_0BP@DFKLHFDI@?$CK?5SRB_FUNCTION_POWER?3?5sleep?51?6?$AA@FNODOBFM@ 0041f8fe     cmddelivery.obj
 0001:0001e91e       ??_C@_0DL@PCKMOFFE@?$CK?5SRB_FUNCTION_POWER?3?5coming?5bac@FNODOBFM@ 0041f91e     cmddelivery.obj
 0001:0001e95a       ??_C@_0CG@NCNALCOB@?$CK?5SRB_FUNCTION_POWER?3?5going?5to?5S@FNODOBFM@ 0041f95a     cmddelivery.obj
 0001:0001e980       ??_C@_0CA@IBGDOHDE@?$CK?5SRB_FUNCTION_POWER?3?5shutdown?6?$AA@FNODOBFM@ 0041f980     cmddelivery.obj
 0001:0001e9a0       ??_C@_0CD@NOANDIPK@?$CK?5SRB_FUNCTION_POWER?3?5shutdownOf@FNODOBFM@ 0041f9a0     cmddelivery.obj
 0001:0001e9c4       ??_C@_0BO@KPPCGIPP@?$CK?5SRB_FUNCTION_POWER?3?5reboot?6?$AA@FNODOBFM@ 0041f9c4     cmddelivery.obj
 0001:0001e9e2       ??_C@_0BJ@NDPKABON@entering?5AdapterControl?6?$AA@FNODOBFM@ 0041f9e2     cmdproc.obj
 0001:0001e9fc       ??_C@_0CF@FDIANAIH@?$CK?5?9?5AdapterControl?3?5ScsiStopAdap@FNODOBFM@ 0041f9fc     cmdproc.obj
 0001:0001ea22       ??_C@_0FJ@DLLPOCIO@?$CK?5?9?5AdapterControl?3?5ScsiStopAdap@FNODOBFM@ 0041fa22     cmdproc.obj
 0001:0001ea7c       ??_C@_0DK@JIECJOFO@?$CK?5Set?5pInitStruct?9?$DONoOfMsiVector@FNODOBFM@ 0041fa7c     cmdproc.obj
 0001:0001eab6       ??_C@_0HA@BIJAMPMG@?$CK?5?9?5AdapterControl?3?5ScsiSetBootC@FNODOBFM@ 0041fab6     cmdproc.obj
 0001:0001eb26       ??_C@_0DL@CMAPNHGC@?$CK?5?9?5AdapterControl?3?5ScsiSetBootC@FNODOBFM@ 0041fb26     cmdproc.obj
 0001:0001eb62       ??_C@_0DI@IPKKLNPP@?$CK?5?9?5AdapterControl?3?5ScsiSetBootC@FNODOBFM@ 0041fb62     cmdproc.obj
 0001:0001eb9a       ??_C@_0HE@CIFLMEO@?$CK?5?9?5AdapterControl?3?5ScsiSetRunni@FNODOBFM@ 0041fb9a     cmdproc.obj
 0001:0001ec0e       ??_C@_0CI@NDPGKLNN@?$CK?5?9?5AdapterControl?3?5ScsiRestartA@FNODOBFM@ 0041fc0e     cmdproc.obj
 0001:0001ec36       ??_C@_0CM@CNGCOMHH@?$CK?5Before?5checking?5Adapter?5Health@FNODOBFM@ 0041fc36     cmdproc.obj
 0001:0001ec62       ??_C@_0BF@GMFKAGLA@?$CK?$CK?5BlinLed?5Code?3?5?$CFx?6?$AA@FNODOBFM@ 0041fc62     cmdproc.obj
 0001:0001ec78       ??_C@_0DM@EBNPFHJD@?$CK?5set?5timer?5to?5check?5the?5FW?5stat@FNODOBFM@ 0041fc78     cmdproc.obj
 0001:0001ecb4       ??_C@_0CM@LGOLDMAP@?$CK?5leaving?5AdapterControl?5Routine@FNODOBFM@ 0041fcb4     cmdproc.obj
 0001:0001ece0       ??_C@_0EF@MIBINBLP@?$CK?5Hw?5Soft?5Reset?5Set?5Timer?0?5leavi@FNODOBFM@ 0041fce0     cmdproc.obj
 0001:0001ed26       ??_C@_0CG@MHIDKAIN@?$CK?5HW?5Soft?5Reset?0?5Set?5Timer?0?5line@FNODOBFM@ 0041fd26     cmdproc.obj
 0001:0001ed4c       ??_C@_0IF@DDPMHFDG@?$CK?5SMNormalModeInitAdapter?5failed@FNODOBFM@ 0041fd4c     cmdproc.obj
 0001:0001edd2       ??_C@_0IE@BILJPPDJ@?$CK?5SMNormalModeInitAdapter?5failed@FNODOBFM@ 0041fdd2     cmdproc.obj
 0001:0001ee56       ??_C@_0CO@CEANCDOF@?$CK?5?9?5AdapterControl?3?5Reset?5HostRR@FNODOBFM@ 0041fe56     cmdproc.obj
 0001:0001ee84       ??_C@_0CN@OHJICFOG@?$CK?5?9?5AdapterControl?3?5ScsiQuery?5wi@FNODOBFM@ 0041fe84     cmdproc.obj
 0001:0001eeb2       ??_C@_0DA@CMHNEFAA@?$CK?5?9?5AdapterControl?3?5ScsiQuery?5WI@FNODOBFM@ 0041feb2     cmdproc.obj
 0001:0001eee2       ??_C@_0DB@DKFDCCOB@?$CK?5Unsupported?5AdapterControl?5cod@FNODOBFM@ 0041fee2     cmdproc.obj
 0001:0001ef14       ??_C@_0BI@MBKDPNLO@leaving?5AdapterControl?6?$AA@FNODOBFM@ 0041ff14     cmdproc.obj
 0001:0001ef2c       ??_C@_0CO@NKBJPPMA@?$CK?5buildio?3?5LBA?5OUT?5OF?5RANGE?0?5sen@FNODOBFM@ 0041ff2c     cmdproc.obj
 0001:0001ef5a       ??_C@_0FN@LKLFGDKL@?$CK?5buildio?3?5LBA?5OUT?5OF?5RANGE?0?5sen@FNODOBFM@ 0041ff5a     cmdproc.obj
 0001:0001efb8       ??_C@_0FA@MOKLGDID@?$CK?5buildio?3?5LBA?5OUT?5OF?5RANGE?0?5sen@FNODOBFM@ 0041ffb8     cmdproc.obj
 0001:0001f008       ??_C@_0GA@IGOANHED@?$CK?5buildio?3?5LBA?5OUT?5OF?5RANGE?0?5sen@FNODOBFM@ 00420008     cmdproc.obj
 0001:0001f068       ??_C@_07MPDDHOMN@CSMIALL?$AA@FNODOBFM@ 00420068     ioctl.obj
 0001:0001f070       ??_C@_07OODOBGKD@CSMIARY?$AA@FNODOBFM@ 00420070     ioctl.obj
 0001:0001f078       ??_C@_07PAKBHMBE@CSMISAS?$AA@FNODOBFM@ 00420078     ioctl.obj
 0001:0001f080       ??_C@_07BHCKAAPP@CSMIPHY?$AA@FNODOBFM@ 00420080     ioctl.obj
 0001:0001f088       ??_C@_0CF@JOCBDLKJ@?$CK?5Allocate?5big?5IOCTL?5buffer?5fail@FNODOBFM@ 00420088     ioctl.obj
 0001:0001f0ae       ??_C@_0DF@CHPLNPBM@?$CK?5ProcessIoctl?3?5Internal?5Print?5B@FNODOBFM@ 004200ae     ioctl.obj
 0001:0001f0e4       ??_C@_0CE@NGAHOGLJ@?$CK?5ProcessIoctl?3?5private?5cdb?8s?5he@FNODOBFM@ 004200e4     ioctl.obj
 0001:0001f108       ??_C@_0CH@HPKPAOCF@?$CK?5ProcessIoctl?3?5DBG_IO_TRACE?5fla@FNODOBFM@ 00420108     ioctl.obj
 0001:0001f130       ??_C@_0CK@OFFABCEM@?$CK?5ProcessIoctl?3?5DBG_IOCTL_TRACE?5@FNODOBFM@ 00420130     ioctl.obj
 0001:0001f15a       ??_C@_0CM@CGIIOCGI@?$CK?5ProcessIoctl?3?5DBG_CLUSTER_TRAC@FNODOBFM@ 0042015a     ioctl.obj
 0001:0001f186       ??_C@_0CI@LPOJHEHM@?$CK?5ProcessIoctl?3?5DBG_ISR_TRACE?5fl@FNODOBFM@ 00420186     ioctl.obj
 0001:0001f1ae       ??_C@_0DC@NOLFHCLF@?$CK?5ProcessIoctl?3?5DBG_IO_FUNC_ENTR@FNODOBFM@ 004201ae     ioctl.obj
 0001:0001f1e0       ??_C@_0DE@PFEFFOBG@?$CK?5ProcessIoctl?3?5DBG_INIT_FUNC_EN@FNODOBFM@ 004201e0     ioctl.obj
 0001:0001f214       ??_C@_0DF@DPLBBPBM@?$CK?5ProcessIoctl?3?5DBG_IOCTL_FUNC_E@FNODOBFM@ 00420214     ioctl.obj
 0001:0001f24a       ??_C@_0CL@GAIHEBC@?$CK?5ProcessIoctl?3?5DBG_IO_TRACE?5fla@FNODOBFM@ 0042024a     ioctl.obj
 0001:0001f276       ??_C@_0CO@NGOEBBKH@?$CK?5ProcessIoctl?3?5DBG_IOCTL_TRACE?5@FNODOBFM@ 00420276     ioctl.obj
 0001:0001f2a4       ??_C@_0DA@HPMIGAD@?$CK?5ProcessIoctl?3?5DBG_CLUSTER_TRAC@FNODOBFM@ 004202a4     ioctl.obj
 0001:0001f2d4       ??_C@_0CM@NECMPDIP@?$CK?5ProcessIoctl?3?5DBG_ISR_TRACE?5fl@FNODOBFM@ 004202d4     ioctl.obj
 0001:0001f300       ??_C@_0DG@PHFPGNCH@?$CK?5ProcessIoctl?3?5DBG_IO_FUNC_ENTR@FNODOBFM@ 00420300     ioctl.obj
 0001:0001f336       ??_C@_0DI@CBNGHMLF@?$CK?5ProcessIoctl?3?5DBG_INIT_FUNC_EN@FNODOBFM@ 00420336     ioctl.obj
 0001:0001f36e       ??_C@_0DJ@DEFCHEDB@?$CK?5ProcessIoctl?3?5DBG_IOCTL_FUNC_E@FNODOBFM@ 0042036e     ioctl.obj
 0001:0001f3a8       ??_C@_0CC@ELKJFKAD@?$CK?5ProcessIoctl?3?5DebugFlags?3?50x?$CFx@FNODOBFM@ 004203a8     ioctl.obj
 0001:0001f3ca       ??_C@_0DI@PNEPHAGL@?$CK?5Set?5pInitStruct?9?$DONoOfMsiVector@FNODOBFM@ 004203ca     ioctl.obj
 0001:0001f402       ??_C@_0DF@KDDHBOCK@?$CK?5when?5back?5from?5IOP_RESET?0?5we?5w@FNODOBFM@ 00420402     ioctl.obj
 0001:0001f438       ??_C@_0DO@IBFHJCIJ@?$CK?5IOP?5RESET?5is?5done?5in?5ProcessIo@FNODOBFM@ 00420438     ioctl.obj
 0001:0001f476       ??_C@_0DN@EJCEJBIF@?$CK?5IOP?5RESET?5failed?5in?5ProcessIoc@FNODOBFM@ 00420476     ioctl.obj
 0001:0001f4b4       ??_C@_0CF@GENCHGED@?$CK?5ProcessIoctl?3?5coalescing?5disab@FNODOBFM@ 004204b4     ioctl.obj
 0001:0001f4da       ??_C@_0CE@KOEFFOB@?$CK?5ProcessIoctl?3?5coalescing?5enabl@FNODOBFM@ 004204da     ioctl.obj
 0001:0001f4fe       ??_C@_0GG@KLCLOEBM@?$CK?5ProcessIoctl?3?5Get?5a?5request?5fo@FNODOBFM@ 004204fe     ioctl.obj
 0001:0001f564       ??_C@_0IA@OEPDMML@?$CK?5ProcessIoctl?3?5Get?5a?5request?5fo@FNODOBFM@ 00420564     ioctl.obj
 0001:0001f5e4       ??_C@_0GG@JMGDPGEE@?$CK?5ProcessIoctl?3?5Get?5a?5request?5fo@FNODOBFM@ 004205e4     ioctl.obj
 0001:0001f64a       ??_C@_0IA@HMGAPIGO@?$CK?5ProcessIoctl?3?5Get?5a?5request?5fo@FNODOBFM@ 0042064a     ioctl.obj
 0001:0001f6ca       ??_C@_0DH@GFOJOHEG@?$CK?5ProcessIoctl?3?5TTYPE_CHANGE_IO_@FNODOBFM@ 004206ca     ioctl.obj
 0001:0001f702       ??_C@_0CN@FFFLABJM@?$CK?5ProcessIoctl?3?5AIF?5commands?5pri@FNODOBFM@ 00420702     ioctl.obj
 0001:0001f730       ??_C@_0CO@EKDJMEJG@?$CK?5ProcessIoctl?3?5AIF?5commands?5pri@FNODOBFM@ 00420730     ioctl.obj
 0001:0001f75e       ??_C@_0CP@DNDOBHJJ@?$CK?5ProcessIoctl?3?5synch?5commands?5p@FNODOBFM@ 0042075e     ioctl.obj
 0001:0001f78e       ??_C@_0DA@DKDLFFAP@?$CK?5ProcessIoctl?3?5synch?5commands?5p@FNODOBFM@ 0042078e     ioctl.obj
 0001:0001f7be       ??_C@_0DD@OCMBIILM@?$CK?5ProcessIoctl?3?5RUN_CODE_IN_SPEC@FNODOBFM@ 004207be     ioctl.obj
 0001:0001f7f2       ??_C@_0FD@PBJMMHDI@?$CK?5ProcessIoctl?3?5RUN_CODE_IN_SPEC@FNODOBFM@ 004207f2     ioctl.obj
 0001:0001f846       ??_C@_0EG@IJGFKELB@?$CK?5ProcessIoctl?3?5bus?$DN?$CFd?0?5target?$DN?$CF@FNODOBFM@ 00420846     ioctl.obj
 0001:0001f88c       ??_C@_0GB@LAAKBHJK@?$CK?5ProcessIoctl?3?5wrong?5parameters@FNODOBFM@ 0042088c     ioctl.obj
 0001:0001f8ee       ??_C@_0DA@LCPJHFEI@?$CK?5ProcessIoctl?3?5Max?5Data?5Transfe@FNODOBFM@ 004208ee     ioctl.obj
 0001:0001f91e       ??_C@_0CE@DJCKDJAF@?$CK?5ProcessIoctl?3?5Max?5SG?5items?3?50x@FNODOBFM@ 0042091e     ioctl.obj
 0001:0001f942       ??_C@_0BF@JHMLOOKE@?$CK?5outstanding?5IO?3?$CFd?6?$AA@FNODOBFM@ 00420942     ioctl.obj
 0001:0001f958       ??_C@_0BO@MJJJDCNP@?$CK?5Coalescing?5Q?4?5CalledCnt?3?$CFd?6?$AA@FNODOBFM@ 00420958     ioctl.obj
 0001:0001f976       ??_C@_0CJ@GBKALEBA@?$CK?5Coalescing?5Q?4?5Beyond8kTransfer@FNODOBFM@ 00420976     ioctl.obj
 0001:0001f9a0       ??_C@_0CJ@OEJKDMEF@?$CK?5Coalescing?5Q?4?5AcrossStripeBoun@FNODOBFM@ 004209a0     ioctl.obj
 0001:0001f9ca       ??_C@_0CD@JOOBICJM@?$CK?5Coalescing?5Q?4?5RwCmdTypeMixed?3?$CF@FNODOBFM@ 004209ca     ioctl.obj
 0001:0001f9ee       ??_C@_0CD@HLIMFKCF@?$CK?5Coalescing?5Q?4?5SGcntOverLimit?3?$CF@FNODOBFM@ 004209ee     ioctl.obj
 0001:0001fa12       ??_C@_0CF@HPODEDGN@?$CK?5Coalescing?5Q?4?5CmdSizeOverLimit@FNODOBFM@ 00420a12     ioctl.obj
 0001:0001fa38       ??_C@_0CF@HCLMLLN@?$CK?5Coalescing?5Q?4?5DequeueCalledCnt@FNODOBFM@ 00420a38     ioctl.obj
 0001:0001fa5e       ??_C@_0CL@HMCMDMGE@?$CK?5Coalescing?5Q?4?5CallSendFibDirec@FNODOBFM@ 00420a5e     ioctl.obj
 0001:0001fa8a       ??_C@_0BL@BDGJNAIM@?$CK?5Sorting?5Q?4?5CalledCnt?3?$CFd?6?$AA@FNODOBFM@ 00420a8a     ioctl.obj
 0001:0001faa6       ??_C@_0BO@FHMIKIJB@?$CK?5Sorting?5Q?4?5OverlapCase1?3?$CFd?6?$AA@FNODOBFM@ 00420aa6     ioctl.obj
 0001:0001fac4       ??_C@_0BO@NBFMNKDP@?$CK?5Sorting?5Q?4?5OverlapCase2?3?$CFd?6?$AA@FNODOBFM@ 00420ac4     ioctl.obj
 0001:0001fae2       ??_C@_0CK@EPAOGNLF@?$CK?5ProcessIoctl?3?5BUILDIO?5LOOPBACK@FNODOBFM@ 00420ae2     ioctl.obj
 0001:0001fb0c       ??_C@_0CK@DADBMBLL@?$CK?5ProcessIoctl?3?5STARTIO?5LOOPBACK@FNODOBFM@ 00420b0c     ioctl.obj
 0001:0001fb36       ??_C@_0CK@BMBGJMJA@?$CK?5ProcessIoctl?3?5PUSHFIB?5LOOPBACK@FNODOBFM@ 00420b36     ioctl.obj
 0001:0001fb60       ??_C@_0CL@DANMEPHG@?$CK?5ProcessIoctl?3?5BUILDIO?5LOOPBACK@FNODOBFM@ 00420b60     ioctl.obj
 0001:0001fb8c       ??_C@_0CL@NHBLFNNN@?$CK?5ProcessIoctl?3?5STARTIO?5LOOPBACK@FNODOBFM@ 00420b8c     ioctl.obj
 0001:0001fbb8       ??_C@_0CL@HLILIDMA@?$CK?5ProcessIoctl?3?5PUSHFIB?5LOOPBACK@FNODOBFM@ 00420bb8     ioctl.obj
 0001:0001fbe4       ??_C@_0DB@MDNCKDFE@?$CK?5ProcessIoctl?3?5Simulate?5SCSI?5sm@FNODOBFM@ 00420be4     ioctl.obj
 0001:0001fc16       ??_C@_0EC@KMBGJBEG@?$CK?5ProcessIoctl?3?5Simulate?5FW?5Targ@FNODOBFM@ 00420c16     ioctl.obj
 0001:0001fc58       ??_C@_0BI@COAKNOP@?$CK?5?9?5IOCTL?5MESSAGE?3?5?$CFs?5?6?$AA@FNODOBFM@ 00420c58     ioctl.obj
 0001:0001fc70       ??_C@_0BP@PHOOCPMJ@?$CK?5?9?5IOCTL?3?5FSAMPCTL_RESET_IOP?6?$AA@FNODOBFM@ 00420c70     ioctl.obj
 0001:0001fc90       ??_C@_0CE@ONNDCLIE@FSAMPCTL_RESET_IOP?5?3?5ResetFlag?5?$CF@FNODOBFM@ 00420c90     ioctl.obj
 0001:0001fcb4       ??_C@_0CN@OOAKPBJA@FSAMPCTL_RESET_IOP?3?5IOP?5Reset?5On@FNODOBFM@ 00420cb4     ioctl.obj
 0001:0001fce2       ??_C@_0CP@PMFIDFBA@?$CK?5IOP?5RESET?5is?5done?5in?5ProcessIo@FNODOBFM@ 00420ce2     ioctl.obj
 0001:0001fd12       ??_C@_0EB@EJNKCDGF@?$CK?5IOP?5RESET?5failed?5in?5ProcessIoc@FNODOBFM@ 00420d12     ioctl.obj
 0001:0001fd54       ??_C@_0DB@GLCCJBC@FSAMPCTL_RESET_IOP?3?5HW?5Soft?5Rese@FNODOBFM@ 00420d54     ioctl.obj
 0001:0001fd86       ??_C@_0DI@EHOOKHPF@?$CK?5when?5back?5from?5HWSOFT_RESET?0?5w@FNODOBFM@ 00420d86     ioctl.obj
 0001:0001fdbe       ??_C@_0DN@BHCOMBAH@?$CK?5set?5timer?5to?5check?5the?5FW?5stat@FNODOBFM@ 00420dbe     ioctl.obj
 0001:0001fdfc       ??_C@_0DD@GMMMAFI@?$CK?5HW?5SOFT?5RESET?5is?5done?5in?5Proce@FNODOBFM@ 00420dfc     ioctl.obj
 0001:0001fe30       ??_C@_0EF@IPKPNMPC@?$CK?5HW?5SOFT?5RESET?5failed?5in?5Proces@FNODOBFM@ 00420e30     ioctl.obj
 0001:0001fe76       ??_C@_0EN@MGMHDFPF@FSAMPCTL_RESET_IOP?3?5IOP?5Reset?5Fo@FNODOBFM@ 00420e76     ioctl.obj
 0001:0001fec4       ??_C@_0DC@MOKOJMEO@?$CK?5HW?5IOP?5RESET?5is?5done?5in?5Proces@FNODOBFM@ 00420ec4     ioctl.obj
 0001:0001fef6       ??_C@_0DO@IOLDEEBK@ProcessIoctl?5FSAMPCTL_RESET_IOP?0@FNODOBFM@ 00420ef6     ioctl.obj
 0001:0001ff34       ??_C@_0L@BGLGDCOP@archba?4sys?$AA@FNODOBFM@ 00420f34     ioctl.obj
 0001:0001ff40       ??_C@_0CA@HJMENHI@Adaptec?5SAS?5HBA?5Storport?5Driver?$AA@FNODOBFM@ 00420f40     ioctl.obj
 0001:0001ff60       ??_C@_0DJ@MIENLJJJ@OMR?5value?5in?5Check?5Adapter?5Healt@FNODOBFM@ 00420f60     comm.obj
 0001:0001ff9a       ??_C@_0EJ@PCHGGBBF@?$CK?5ProcessAif?3?5request?5timer?5for?5@FNODOBFM@ 00420f9a     comm.obj
 0001:0001ffe4       ??_C@_0BL@NHJOLJMJ@AIF?5EVENT?5?$CIThor?$CJ?3?5HotPlug?6?$AA@FNODOBFM@ 00420fe4     comm.obj
 0001:00020000       ??_C@_0CD@EMEGIPDM@AIF?5EVENT?5?$CIThor?$CJ?3?5Hardware?5chang@FNODOBFM@ 00421000     comm.obj
 0001:00020024       ??_C@_0DC@LGHJMKLE@AIF?5EVENT?5?$CIThor?$CJ?3?5Physical?5Devic@FNODOBFM@ 00421024     comm.obj
 0001:00020056       ??_C@_0DB@CEOPCOBC@AIF?5EVENT?5?$CIThor?$CJ?3?5Logical?5Device@FNODOBFM@ 00421056     comm.obj
 0001:00020088       ??_C@_0DC@PEAKFMNI@AIF?5EVENT?5?$CIThor?$CJ?3?5FW?5IO?5bypass?5s@FNODOBFM@ 00421088     comm.obj
 0001:000200ba       ??_C@_0DK@MABGHGOH@AIF?5EVENT?5?$CIThor?$CJ?3?5FW?5IO?5bypass?5c@FNODOBFM@ 004210ba     comm.obj
 0001:000200f4       ??_C@_0CP@MLBBLAGJ@AIF?5EVENT?5?$CIThor?$CJ?3?5Not?5a?5recogniz@FNODOBFM@ 004210f4     comm.obj
 0001:00020124       ??_C@_0DL@CJKFCOBN@?$CK?5ProcessAif?3?5request?5timer?5to?5s@FNODOBFM@ 00421124     comm.obj
 0001:00020160       ??_C@_0CH@PCLLKGG@?$CK?5ProcessAif?3?5Physical?5Drives?5sc@FNODOBFM@ 00421160     comm.obj
 0001:00020188       ??_C@_0DK@NNFHFOND@?$CK?5ProcessAif?3?5request?5timer?5to?5s@FNODOBFM@ 00421188     comm.obj
 0001:000201c2       ??_C@_0CG@CDKKDOHL@?$CK?5ProcessAif?3?5Logical?5Drives?5sca@FNODOBFM@ 004211c2     comm.obj
 0001:000201e8       ??_C@_0EO@LMDDDIBO@?$CK?5RestoreBMIC15Srb?3?5QD?5limitatio@FNODOBFM@ 004211e8     comm.obj
 0001:00020236       ??_C@_0EI@IBBGKNJF@?$CK?5ProcessNormalFib?9Set?5QD?54?5HBA?5@FNODOBFM@ 00421236     comm.obj
 0001:0002027e       ??_C@_0CG@IPLFJLPL@Smart?5HBA?5Scsi?5response?5Status?5?$DN@FNODOBFM@ 0042127e     comm.obj
 0001:000202a4       ??_C@_0DO@HNDDHFGA@?5HBA?5Error?5HBA_MODE_DISABLED?5Srb@FNODOBFM@ 004212a4     comm.obj
 0001:000202e2       ??_C@_0DA@CPGPCCBA@?5HBA?5Error?5code?5?$CFx?5For?5Path?5ID?5?$CF@FNODOBFM@ 004212e2     comm.obj
 0001:00020312       ??_C@_0FA@CPHJLELC@?5HBA?5Error?5SCSI_COMPL_TRANSL_STA@FNODOBFM@ 00421312     comm.obj
 0001:00020362       ??_C@_0FE@JFIIIBKF@?5HBA?5Error?5SCSI_COMPL_TRANSL_STA@FNODOBFM@ 00421362     comm.obj
 0001:000203b6       ??_C@_0EO@DHIENLOG@?5HBA?5Error?3?5Length?5from?5OS?$CI0x?$CFx?$CJ@FNODOBFM@ 004213b6     comm.obj
 0001:00020404       ??_C@_0HP@ECKDIFKN@?5HBA?5Error?3?5hbaCmd?9?$DOdata_length?$CI@FNODOBFM@ 00421404     comm.obj
 0001:00020484       ??_C@_0FK@IBAGLEPN@?5HBA?5Error?5SCSI_COMPL_TRANSL_STA@FNODOBFM@ 00421484     comm.obj
 0001:000204de       ??_C@_0FJ@DMCDLFNM@?5HBA?5Error?5SCSI_COMPL_TRANSL_STA@FNODOBFM@ 004214de     comm.obj
 0001:00020538       ??_C@_0EP@JHLDIODO@?$CK?5NO?5ERROR?5handling?5for?5pHbaResp@FNODOBFM@ 00421538     comm.obj
 0001:00020588       ??_C@_0CG@PJJANG@TMF?5Function?5Completed?5Successfu@FNODOBFM@ 00421588     comm.obj
 0001:000205ae       ??_C@_0FJ@OIALMBME@?$CK?5NO?5ERROR?5handling?5for?5pHbaResp@FNODOBFM@ 004215ae     comm.obj
 0001:00020608       ??_C@_1BI@BHAHBMFJ@?$AAM?$AAo?$AAf?$AAR?$AAe?$AAs?$AAo?$AAu?$AAr?$AAc?$AAe?$AA?$AA@FNODOBFM@ 00421608     wmi.obj
 0001:00020620       ??_C@_1BK@EPHGJNJ@?$AAS?$AAc?$AAs?$AAi?$AAM?$AAi?$AAn?$AAi?$AAP?$AAo?$AAr?$AAt?$AA?$AA@FNODOBFM@ 00421620     scsiwmi:wmilib.obj
 0002:00000000       __imp__memset              00422000     ntoskrnl:ntoskrnl.exe
 0002:00000004       __imp___aulldvrm           00422004     ntoskrnl:ntoskrnl.exe
 0002:00000008       __imp__ExSystemTimeToLocalTime@8 00422008     ntoskrnl:ntoskrnl.exe
 0002:0000000c       __imp__RtlTimeToTimeFields@8 0042200c     ntoskrnl:ntoskrnl.exe
 0002:00000010       __imp___alldiv             00422010     ntoskrnl:ntoskrnl.exe
 0002:00000014       __imp___allmul             00422014     ntoskrnl:ntoskrnl.exe
 0002:00000018       __imp___aulldiv            00422018     ntoskrnl:ntoskrnl.exe
 0002:0000001c       __imp___aullshr            0042201c     ntoskrnl:ntoskrnl.exe
 0002:00000020       \177ntoskrnl_NULL_THUNK_DATA 00422020     ntoskrnl:ntoskrnl.exe
 0002:00000024       __imp__StorPortGetPhysicalAddress@16 00422024     storport:storport.sys
 0002:00000028       __imp__StorPortPause@8     00422028     storport:storport.sys
 0002:0000002c       __imp__StorPortNotification 0042202c     storport:storport.sys
 0002:00000030       __imp__StorPortStallExecution@4 00422030     storport:storport.sys
 0002:00000034       __imp__StorPortReadRegisterUchar@8 00422034     storport:storport.sys
 0002:00000038       __imp__StorPortReadRegisterUlong@8 00422038     storport:storport.sys
 0002:0000003c       __imp__StorPortReadRegisterBufferUchar@16 0042203c     storport:storport.sys
 0002:00000040       __imp__StorPortWriteRegisterUlong@12 00422040     storport:storport.sys
 0002:00000044       __imp__StorPortWriteRegisterBufferUlong@16 00422044     storport:storport.sys
 0002:00000048       __imp__StorPortMoveMemory@12 00422048     storport:storport.sys
 0002:0000004c       __imp__StorPortDebugPrint  0042204c     storport:storport.sys
 0002:00000050       __imp__StorPortGetDeviceBase@28 00422050     storport:storport.sys
 0002:00000054       __imp__StorPortWriteRegisterBufferUchar@16 00422054     storport:storport.sys
 0002:00000058       __imp__StorPortResume@4    00422058     storport:storport.sys
 0002:0000005c       __imp__StorPortExtendedFunction 0042205c     storport:storport.sys
 0002:00000060       __imp__StorPortInitialize@16 00422060     storport:storport.sys
 0002:00000064       __imp__StorPortFreeDeviceBase@8 00422064     storport:storport.sys
 0002:00000068       __imp__StorPortGetBusData@24 00422068     storport:storport.sys
 0002:0000006c       __imp__StorPortGetUncachedExtension@12 0042206c     storport:storport.sys
 0002:00000070       __imp__StorPortSetDeviceQueueDepth@20 00422070     storport:storport.sys
 0002:00000074       __imp__StorPortQuerySystemTime@4 00422074     storport:storport.sys
 0002:00000078       __imp__StorPortPauseDevice@20 00422078     storport:storport.sys
 0002:0000007c       __imp__StorPortResumeDevice@16 0042207c     storport:storport.sys
 0002:00000080       __imp__StorPortBusy@8      00422080     storport:storport.sys
 0002:00000084       __imp__StorPortGetScatterGatherList@8 00422084     storport:storport.sys
 0002:00000088       __imp__ScsiPortMoveMemory@12 00422088     storport:storport.sys
 0002:0000008c       \177storport_NULL_THUNK_DATA 0042208c     storport:storport.sys
 0002:00000128       _RevCompareTable           00422128     revision.obj
 0002:00000228       _RevCompareTableLength     00422228     revision.obj
 0002:000002ec       ??_C@_08HNOCAICB@Adaptec?5?$AA@ 004222ec     archba.obj
 0002:000002f8       ??_C@_04ODJNANJC@9005?$AA@ 004222f8     archba.obj
 0002:00000300       ??_C@_04EKJHPGNA@0285?$AA@ 00422300     archba.obj
 0002:00000308       ??_C@_04GBLKKFBD@0286?$AA@ 00422308     archba.obj
 0002:00000310       ??_C@_04PPDJIIJN@0288?$AA@ 00422310     archba.obj
 0002:00000318       ??_C@_04LPGNDNED@028b?$AA@ 00422318     archba.obj
 0002:00000320       ??_C@_04KGHGAMAC@028c?$AA@ 00422320     archba.obj
 0002:00000328       ??_C@_04OJDHJKMF@028d?$AA@ 00422328     archba.obj
 0002:00000330       ??_C@_0BB@BOPAMEAE@ARC?9HBA?5?5?5?5?5?5?5?5?5?$AA@ 00422330     archba.obj
 0002:00000344       ??_C@_06DFBHEALI@AACAPI?$AA@ 00422344     archba.obj
 0002:00000470       __load_config_used         00422470     BufferOverflowFastFailK:loadcfg.obj
 0002:00000500       ___safe_se_handler_table   00422500     <linker-defined>
 0003:00000000       _gDebugFlags               00423000     arcdebug.obj
 0003:00000008       _gNativeModeAdapters       00423008     archba.obj
 0003:000001b8       _gNumNativeModeAdapters    004231b8     archba.obj
 0003:000001bc       _gARCProductId             004231bc     archba.obj
 0003:000001c0       _gARCApiId                 004231c0     archba.obj
 0003:000001c4       _gARCOEMFlags              004231c4     archba.obj
 0003:000001c8       _gARCSASRxSubsystemInfo    004231c8     archba.obj
 0003:00000350       _gARCSASRktSubsystemInfo   00423350     archba.obj
 0003:00000388       _gARCSASArkSubsystemInfo   00423388     archba.obj
 0003:000003a0       _gARCSASPMCSubsystemInfo   004233a0     archba.obj
 0003:00000520       _gARCVendor                00423520     arcinit.obj
 0003:00000524       _gAdapterGuid              00423524     wmi.obj
 0003:00000534       _gIoChannelGuid            00423534     wmi.obj
 0003:00000544       _gDiskArrayGuid            00423544     wmi.obj
 0003:00000554       _gPhysicalDiskGuid         00423554     wmi.obj
 0003:00000564       _gAdapterMethodGuid        00423564     wmi.obj
 0003:00000574       ___security_cookie         00423574     BufferOverflowFastFailK:gs_support.obj
 0003:00000578       ___security_cookie_complement 00423578     BufferOverflowFastFailK:gs_support.obj
 0003:000005b0       _gLatency                  004235b0     arcinit.obj
 0003:000005b4       _gLoopbackInPushFib        004235b4     arcinit.obj
 0003:000005b8       _gTraceContext             004235b8     arcinit.obj
 0003:000005bc       _gAdapterAddCount          004235bc     arcinit.obj
 0003:00000640       _gAdapterTable             00423640     <common>
 0003:00000740       _gDriverObject             00423740     <common>
 0004:00000006       ___security_init_cookie    00424006 f   BufferOverflowFastFailK:gs_support.obj
 0004:00000030       __IMPORT_DESCRIPTOR_ntoskrnl 00424030     ntoskrnl:ntoskrnl.exe
 0004:00000044       __IMPORT_DESCRIPTOR_storport 00424044     storport:storport.sys
 0004:00000058       __NULL_IMPORT_DESCRIPTOR   00424058     ntoskrnl:ntoskrnl.exe

 entry point at        0001:00018a70

 Static symbols

 0000:fffd8000       .debug$S                   00400000     storport:storport.sys
 0000:fffd8000       .debug$S                   00400000     storport:storport.sys
 0000:fffd8000       .debug$S                   00400000     storport:storport.sys
 0000:fffd8000       .debug$S                   00400000     storport:storport.sys
 0000:fffd8000       .debug$S                   00400000     storport:storport.sys
 0000:fffd8000       .debug$S                   00400000     storport:storport.sys
 0000:fffd8000       .debug$S                   00400000     storport:storport.sys
 0000:fffd8000       .debug$S                   00400000     storport:storport.sys
 0000:fffd8000       .debug$S                   00400000     storport:storport.sys
 0000:fffd8000       .debug$S                   00400000     storport:storport.sys
 0000:fffd8000       .debug$S                   00400000     ntoskrnl:ntoskrnl.exe
 0000:fffd8000       .debug$S                   00400000     ntoskrnl:ntoskrnl.exe
 0000:fffd8000       .debug$S                   00400000     ntoskrnl:ntoskrnl.exe
 0000:fffd8000       .debug$S                   00400000     storport:storport.sys
 0000:fffd8000       .debug$S                   00400000     storport:storport.sys
 0000:fffd8000       .debug$S                   00400000     storport:storport.sys
 0000:fffd8000       .debug$S                   00400000     storport:storport.sys
 0000:fffd8000       .debug$S                   00400000     ntoskrnl:ntoskrnl.exe
 0000:fffd8000       .debug$S                   00400000     ntoskrnl:ntoskrnl.exe
 0000:fffd8000       .debug$S                   00400000     ntoskrnl:ntoskrnl.exe
 0000:fffd8000       .debug$S                   00400000     storport:storport.sys
 0000:fffd8000       .debug$S                   00400000     storport:storport.sys
 0000:fffd8000       .debug$S                   00400000     storport:storport.sys
 0000:fffd8000       .debug$S                   00400000     storport:storport.sys
 0000:fffd8000       .debug$S                   00400000     storport:storport.sys
 0000:fffd8000       .debug$S                   00400000     storport:storport.sys
 0000:fffd8000       .debug$S                   00400000     storport:storport.sys
 0000:fffd8000       .debug$S                   00400000     storport:storport.sys
 0000:fffd8000       .debug$S                   00400000     storport:storport.sys
 0000:fffd8000       .debug$S                   00400000     storport:storport.sys
 0000:fffd8000       .debug$S                   00400000     storport:storport.sys
 0000:fffd8000       .debug$S                   00400000     storport:storport.sys
 0000:fffd8000       .debug$S                   00400000     ntoskrnl:ntoskrnl.exe
 0000:fffd8000       .debug$S                   00400000     ntoskrnl:ntoskrnl.exe
 0000:fffd8000       .debug$S                   00400000     storport:storport.sys
 0001:00000fb0       $LN20                      00401fb0     rxdevice.obj
 0001:00003cf8       $LN145                     00404cf8     arcdebug.obj
 0001:00003d10       $LN138                     00404d10     arcdebug.obj
 0001:00003d40       _StrcatLocal@8             00404d40 f   arcdebug.obj
 0001:00003d80       _Strcatc@8                 00404d80 f   arcdebug.obj
 0001:00006980       $LN15                      00407980     arcinit.obj
 0001:0000bb48       $LN38                      0040cb48     arcinit.obj
 0001:0000beb8       $LN52                      0040ceb8     arcinit.obj
 0001:0000c660       $LN191                     0040d660     arcinit.obj
 0001:0000e6f8       $LN146                     0040f6f8     cmddelivery.obj
 0001:0000e720       $LN127                     0040f720     cmddelivery.obj
 0001:0000e7bc       $LN147                     0040f7bc     cmddelivery.obj
 0001:0000e7e0       $LN128                     0040f7e0     cmddelivery.obj
 0001:00010560       $LN151                     00411560     cmddelivery.obj
 0001:00010578       $LN139                     00411578     cmddelivery.obj
 0001:00010cbc       $LN62                      00411cbc     cmdproc.obj
 0001:00011d40       $LN178                     00412d40     cmdproc.obj
 0001:00011d58       $LN159                     00412d58     cmdproc.obj
 0001:00011d80       $LN179                     00412d80     cmdproc.obj
 0001:00011d90       $LN160                     00412d90     cmdproc.obj
 0001:0001406c       $LN24                      0041506c     ioctl.obj
 0001:0001409c       $LN19                      0041509c     ioctl.obj
 0001:000164d8       $LN367                     004174d8     ioctl.obj
 0001:00016518       $LN326                     00417518     ioctl.obj
 0001:0001655c       $LN368                     0041755c     ioctl.obj
 0001:00016570       $LN327                     00417570     ioctl.obj
 0001:00016f90       $LN65                      00417f90     comm.obj
 0001:0001735c       $LN35                      0041835c     comm.obj
 0001:00017378       $LN32                      00418378     comm.obj
 0001:00017da0       $LN191                     00418da0     comm.obj
 0001:00017db4       $LN171                     00418db4     comm.obj
 0001:00018eea       $LN81                      00419eea     scsiwmi:wmilib.obj
 0001:00019130       $$000000                   0041a130     BufferOverflowFastFailK:forceseh.obj
 0002:000000c8       _STORPORT_POFX_ADAPTER_GUID 004220c8     rxdevice.obj
 0002:000000d8       _STORPORT_POFX_LUN_GUID    004220d8     rxdevice.obj
 0002:000000e8       _STORPORT_DEVICEOPERATION_SECURE_REPROVISION_GUID 004220e8     rxdevice.obj
 0002:000000f8       _STORPORT_POFX_ADAPTER_GUID 004220f8     revision.obj
 0002:00000108       _STORPORT_POFX_LUN_GUID    00422108     revision.obj
 0002:00000118       _STORPORT_DEVICEOPERATION_SECURE_REPROVISION_GUID 00422118     revision.obj
 0002:0000022c       _STORPORT_POFX_ADAPTER_GUID 0042222c     helpers.obj
 0002:0000023c       _STORPORT_POFX_LUN_GUID    0042223c     helpers.obj
 0002:0000024c       _STORPORT_DEVICEOPERATION_SECURE_REPROVISION_GUID 0042224c     helpers.obj
 0002:0000025c       _STORPORT_POFX_ADAPTER_GUID 0042225c     arcdebug.obj
 0002:0000026c       _STORPORT_POFX_LUN_GUID    0042226c     arcdebug.obj
 0002:0000027c       _STORPORT_DEVICEOPERATION_SECURE_REPROVISION_GUID 0042227c     arcdebug.obj
 0002:0000028c       _STORPORT_POFX_ADAPTER_GUID 0042228c     timer.obj
 0002:0000029c       _STORPORT_POFX_LUN_GUID    0042229c     timer.obj
 0002:000002ac       _STORPORT_DEVICEOPERATION_SECURE_REPROVISION_GUID 004222ac     timer.obj
 0002:000002bc       _STORPORT_POFX_ADAPTER_GUID 004222bc     archba.obj
 0002:000002cc       _STORPORT_POFX_LUN_GUID    004222cc     archba.obj
 0002:000002dc       _STORPORT_DEVICEOPERATION_SECURE_REPROVISION_GUID 004222dc     archba.obj
 0002:0000034c       _STORPORT_POFX_ADAPTER_GUID 0042234c     arcinit.obj
 0002:0000035c       _STORPORT_POFX_LUN_GUID    0042235c     arcinit.obj
 0002:0000036c       _STORPORT_DEVICEOPERATION_SECURE_REPROVISION_GUID 0042236c     arcinit.obj
 0002:0000037c       _STORPORT_POFX_ADAPTER_GUID 0042237c     cmddelivery.obj
 0002:0000038c       _STORPORT_POFX_LUN_GUID    0042238c     cmddelivery.obj
 0002:0000039c       _STORPORT_DEVICEOPERATION_SECURE_REPROVISION_GUID 0042239c     cmddelivery.obj
 0002:000003ac       _STORPORT_POFX_ADAPTER_GUID 004223ac     cmdproc.obj
 0002:000003bc       _STORPORT_POFX_LUN_GUID    004223bc     cmdproc.obj
 0002:000003cc       _STORPORT_DEVICEOPERATION_SECURE_REPROVISION_GUID 004223cc     cmdproc.obj
 0002:000003dc       _STORPORT_POFX_ADAPTER_GUID 004223dc     ioctl.obj
 0002:000003ec       _STORPORT_POFX_LUN_GUID    004223ec     ioctl.obj
 0002:000003fc       _STORPORT_DEVICEOPERATION_SECURE_REPROVISION_GUID 004223fc     ioctl.obj
 0002:0000040c       _STORPORT_POFX_ADAPTER_GUID 0042240c     comm.obj
 0002:0000041c       _STORPORT_POFX_LUN_GUID    0042241c     comm.obj
 0002:0000042c       _STORPORT_DEVICEOPERATION_SECURE_REPROVISION_GUID 0042242c     comm.obj
 0002:0000043c       _STORPORT_POFX_ADAPTER_GUID 0042243c     wmi.obj
 0002:0000044c       _STORPORT_POFX_LUN_GUID    0042244c     wmi.obj
 0002:0000045c       _STORPORT_DEVICEOPERATION_SECURE_REPROVISION_GUID 0042245c     wmi.obj
 0003:00000004       ?NeedToReadStatus@?1??CheckingFWAfterPowerStateChange@@9@9 00423004     timer.obj
 0003:00000005       ?NeedToCheckMSIX@?1??CheckingFWAfterPowerStateChange@@9@9 00423005     timer.obj
 0003:00000580       ?cccnt@?1??PMCPushMessageUnitQueueFib@@9@9 00423580     rxdevice.obj
 0003:00000584       ?CurrentCmdCode@?1??RxSendSynchCommand@@9@9 00423584     rxdevice.obj
 0003:00000588       ?CalledCnt@?1??CheckFWPulseInCrashDumpMode@@9@9 00423588     timer.obj
 0003:0000058c       ?TimerAge@?1??CheckingFWAfterPowerStateChange@@9@9 0042358c     timer.obj
 0003:00000590       ?DelayCnt4DualFWFlushSoftReset@?1??CheckingFWAfterPowerStateChange@@9@9 00423590     timer.obj
 0003:00000594       ?pSavedDevExt@?1??CheckingFWAfterPowerStateChange@@9@9 00423594     timer.obj
 0003:00000598       ?TimerAge@?1??Reset_IOP_CompletionTimer@@9@9 00423598     timer.obj
 0003:0000059c       ?status@?1??CheckingFWAfterPowerStateChange@@9@9 0042359c     timer.obj
 0003:000005a0       ?NewScanStarted@?1??ConfigureContainersRuntime@@9@9 004235a0     arcinit.obj
 0003:000005a1       ?LoopCount@?1??ConfigureContainersRuntime@@9@9 004235a1     arcinit.obj
 0003:000005a2       ?busChange@?1??ConfigureContainersRuntime@@9@9 004235a2     arcinit.obj
 0003:000005a3       ?initialized@?1??DriverEntry@@9@9 004235a3     arcinit.obj
 0003:000005a4       ?containerCount@?1??ConfigureContainersRuntime@@9@9 004235a4     arcinit.obj
 0003:000005a8       ?pSavedDevExt@?1??ConfigureContainersRuntime@@9@9 004235a8     arcinit.obj
 0003:000005ac       ?SkipSecondSynchCmd@?1??ConfigureContainersRuntime@@9@9 004235ac     arcinit.obj
 0003:000005c0       ?diskInfoResponse@?1??ConfigureContainersRuntime@@9@9 004235c0     arcinit.obj
 0003:00000628       ?ShutdownSent@?1??BuildIo@@9@9 00423628     cmdproc.obj
 0004:0000016e       .idata$6                   0042416e     ntoskrnl:ntoskrnl.exe
 0004:0000040a       .idata$6                   0042440a     storport:storport.sys
 0005:000000d0       $R000000                   004250d0     archba.res
 0005:00000428       $R000358                   00425428     archba.res
